:020000040800F2
:10000000980A00200D020008874500088135000885
:10001000854500088D140008595B000800000000A9
:100020000000000000000000000000008D540008E7
:10003000FD150008000000003B530008A75400080D
:1000400027020008270200082702000827020008EC
:1000500027020008270200082702000827020008DC
:1000600027020008270200082702000827020008CC
:1000700027020008270200082702000827020008BC
:1000800011150008270200082702000827020008AF
:10009000270200082702000827020008270200089C
:1000A000270200080555000827020008270200085B
:1000B00027020008270200082702000891350008DF
:1000C00085350008270200082702000827020008DB
:1000D00015540008F95A00082D5B00084D5B000814
:1000E000270200082702000827020008270200084C
:1000F000270200082702000827020008270200083C
:10010000270200082702000827020008270200082B
:10011000270200082702000827020008270200081B
:10012000270200082702000827020008270200080B
:1001300000F002F800F05AF80AA090E8000C82449F
:100140008344AAF10107DA4501D100F04FF8AFF27C
:10015000090EBAE80F0013F0010F18BFFB1A43F0A5
:1001600001031847C47B0000E47B00000A4410F838
:10017000014B14F00F0508BF10F8015B240908BFFC
:1001800010F8014B6D1E05D010F8013B6D1E01F8F3
:10019000013BF9D1641E03D0641E01F8015BFBD161
:1001A0009142E4D37047000000230024002500267C
:1001B000103A28BF78C1FBD8520728BF30C148BFCA
:1001C0000B607047662907F0D280642900F05280E6
:1001D000002070471FB500F0C1FB04000020002183
:1001E00006F00CF9E0601FBD10B510BD00F0B6FCC4
:1001F0001146FFF7EFFF06F019F800F0D4FC03B446
:10020000FFF7F2FF03BC00F017FD0000094880472C
:1002100009480047FEE7FEE7FEE7FEE7FEE7FEE7E8
:10022000FEE7FEE7FEE7FEE704480549054A064B00
:1002300070470000035500083101000898040020B1
:10024000980A002098060020980600200FB41CB5DC
:10025000074B06AA7B4469460090059800F065FBB1
:100260000020694600F074FB1CBC5DF814FB000024
:10027000F90600002DE9F0410646002410687529B2
:10028000314616A510D0AFF30080002802DA4042B4
:1002900013A507E031688A0701D512A502E04907D6
:1002A00004D511A5012401E0AFF3008000210A224A
:1002B00006F1240709E0B0FBF2FCB0FBF2F302FB0D
:1002C0001C00303078541846491C0028F3D12346CE
:1002D0002A463046BDE8F04100F0B9B80000000001
:1002E0002D0000002B000000200000002DE9F04749
:1002F0004FF0000A89460446C0F820A02046E16875
:100300008847002876D0252806D0D4E901219047D7
:10031000206A401C2062F1E7E168204600258847FA
:10032000C4F81CA006460027C4F818A02A2E09D03D
:10033000304605F0F1FC38B304EB8708303EC8F8CE
:10034000186019E059F8041B204604EB87029161FC
:10035000E1688847012F064618D1E069002820DAB5
:1003600025F020051DE0D8F8180000EB800006EB12
:1003700040003038C8F818002046E1688847064633
:1003800005F0CAFC0028EED1012F0AD02E2E08D18C
:100390002046E16888477F1C0646022F45F020056D
:1003A000C4DBA069002803DA404245F00105A061E2
:1003B000E80701D025F01005B6B1A6F141001928D3
:1003C00002D8203645F400654A463146204625606D
:1003D0004D46FFF7F7FE58B1012806D0ED1D25F078
:1003E000070000F1080989E704E005F1040985E741
:1003F00030468AE7206ABDE8F0874FF0000200B57A
:10040000134694469646203922BFA0E80C50A0E837
:100410000C50B1F12001BFF4F7AF090728BFA0E8E5
:100420000C5048BF0CC05DF804EB890028BF40F8B1
:10043000042B08BF704748BF20F8022B11F0804FF3
:1004400018BF00F8012B70477047704770472DE9BF
:10045000F0470D4699469246044600F1240801688B
:10046000880604D5E06921F01001216000E0012038
:10047000A84201DD471B00E00027A1697A1902EBC1
:100480000900081AA0612078C00602D42046AFF304
:100490000080002608E0D4E901211AF80600904700
:1004A000206A401C761C20624E45F4DB2078C00692
:1004B0000AD52046AFF3008006E0D4E901213020C0
:1004C0009047206A401C2062381EA7F10107F4DC27
:1004D00007E0D4E9012118F805009047206A401C84
:1004E0002062281EA5F10105F3DC2046AFF3008051
:1004F0002078000602D50220BDE8F0870120FBE746
:1005000070472DE9FF4F0C461E464FF0FF378BB06A
:10051000D2E90001DDF860800A908A46C1F30A55ED
:1005200005B93D46002108464FF00000BAF1000F22
:1005300000F4400005DA00EB80004FF4400101EACE
:1005400050004FEA9059B9F1010F00DDB9460A9801
:1005500050EA4A000ED044F61050A5F2FF3545434C
:100560002F14B8F1000F1ED07542291E1EDDC9F1EF
:1005700000021CE0B8F1010F4FF0000001D0302163
:1005800003E0F24305E02154401CB042FBDB30465F
:100590000022002121540B99C1F80880C1E90020F4
:1005A0000FB0BDE8F08FBD1B6D1CDEE74A4600DAD8
:1005B000694206A800F05CFA06AB93E8070003ABBB
:1005C00083E8070050460A9900F03DFB8DE80700DC
:1005D000A0F500501F3800900398002D0ADD42F26C
:1005E0001F014A460844002303A90390684600F00F
:1005F000A6FD09E0A0F500504A461F38002303A9D4
:100600000390684600F0B0FD8DE807000004000C80
:1006100003D04FF0FF30410800E01046B8F1000F62
:1006200003D00022009215461EE0751E05D400F08E
:1006300099F9303262556D1EF9D5B346012208434F
:1006400002D000227F1C04E02078302801D1002253
:100650007F1E002A099784D01DE0112D07DA00F0D3
:1006600081F9303262556D1C50EA0102F5D1084320
:1006700002D00098C8B10EE00021681E05E0235C9E
:10068000625C63542254401E491C8142F7DBAB4636
:10069000A81B401E0990002004F80B000B98099A33
:1006A000C0F80880C0E9002B7AE711264FF0000857
:1006B00057E72DE9F04F88460446D21D22F0070186
:1006C00091B0D1E90001CDE90A0105F001FB024634
:1006D0000B98C00F01D02D2007E02068810701D5BD
:1006E0002B2002E0202101EAC000032A099001D05A
:1006F000072A05DB03464146204600F079F90BE165
:100700002078800601D5E06900E00620B8F1650F89
:10071000814606D0B8F1660F18D0B8F1670F70D1D6
:1007200031E00020B9F1110F009001DB112301E04D
:1007300009F101030AAA01A90CA8FFF7E2FEDDE90D
:100740000C70002609F10105834647E001204B4665
:1007500000904FF000470AAA01A90CA8FFF7D1FEAC
:10076000DDE90DB00C995D46002610B909F10100D4
:100770000D18B9EB050003D4C0F1FF3609F10105EE
:10078000A5EB09002BE0B9F1010F01DA4FF00109E7
:100790000020B9F1110F0090484601DD112300E05F
:1007A00003460AAA01A90CA8FFF7ABFEDDE90C700D
:1007B0004D4600268346207800070AD4AB4500DA70
:1007C0005D4601A8012D04DD411911F8011C3029F5
:1007D00007D04F4502DA17F1040F04DA01208246F0
:1007E0000FE06D1EEEE7002F02DCED1B3E4403E040
:1007F000781CA84200DD7D1CB81B00F1010A4FF0F7
:1008000000472078000703D4AA4501DB4FF0FF3AE8
:100810000021B7F1004F0DF143088DF8431024D0AB
:1008200002202B23002F01DA7F422D230A21021EF2
:10083000A0F1010000DC5FB197FBF1FC97FBF1F246
:1008400001FB1C7C17460CF1300C08F801CDEEE7DB
:10085000A8F1010003702188090501D5452100E0B8
:100860006521A0F1010800F8011C09980FA9A1EB6E
:100870000807FF1D00B10120411901EBEA70A169D1
:100880003844081A401EA0612078C00602D42046D1
:10089000AFF30080099828B1D4E901219047206A7C
:1008A000401C20622078C00622D52046AFF300808D
:1008B0001EE0002E04DBB34502DD01A8805D00E0F0
:1008C0003020D4E901219047206A401C2062761C28
:1008D000AAF101005FEA000A0AD100F03FF8C068FF
:1008E0000168405CD4E901219047206A401C2062E5
:1008F000281EA5F10105DCDC07E0D4E9012118F888
:10090000010B9047206A401C2062381EA7F10107A6
:10091000F3DC2046AFF30080032011B041E6000075
:1009200001694A1C02610878704700B58FB0CDE9B3
:1009300001310021059105497944CDE903101146A3
:100940006846FFF7D3FC0FB000BD0000E5FFFFFFD6
:100950000A6802F8010B0A607047000000487047FF
:100960005804002030B5B0F10A024FEA900E71F140
:1009700000034EEA817EB0EB0E0061EB91014FEA7D
:10098000101E4EEA017E10EB0E0041EB11114FEAF2
:10099000102E4EEA016E10EB0E0041EB11214FEAD2
:1009A000104E4EEA014E10EB0E0041EB1141401883
:1009B00041F100014FEAD00040EA41704FEAD10115
:1009C00010EB80054FEA810444EA907444EB010483
:1009D0006D1944EB0404521BA3414FF0000348BFC0
:1009E0000A3200D530BD401C41F1000130BD00008D
:1009F0002DE9F0411F46044603260168072A01F449
:100A0000006004DB08B116A505E016A503E008B1F7
:100A100015A500E015A521F010002060A069C01EFA
:100A2000A0610FB1401EA0612046AFF300804FB11E
:100A3000D4E9012138469047206A401C2062C01C3E
:100A4000206206E0206AFAE7D4E9012115F8010BDB
:100A50009047761EF8D22046AFF30080BDE8F081C3
:100A60004E414E006E616E00494E4600696E660052
:100A70002DE9F047814616468AB0354878440DC8BE
:100A80008DE80D0032487844801C03AC0DC884E822
:100A90000D0041F69B300844372190FBF1F290FBAA
:100AA000F1F5A5F1800501FB12041B3C02D564425F
:100AB000012000E00020DFF898A080460027FA44DB
:100AC000AAF1BE0A0EE0E0070AD03246684607EBFC
:100AD000470101230AEB810100F046FB8DE8070086
:100AE00064107F1C002CEED1194F7F44AE3F19E0FB
:100AF000E80715D007EB04100DF1180A90E80E0076
:100B00008AE80E00C068F04201D198190890324678
:100B1000012306A903A800F027FB03AB83E8070025
:100B20006D10641C002DE3D14FF00103324669467D
:100B3000B8F1000F03A802D000F001FB01E000F0C3
:100B400013FBC9E90001C9F808200AB0BDE8F08725
:100B50009072000000487047380400207546FFF787
:100B6000F9FFAE4605006946534620F0070085466A
:100B700018B020B5FFF758FBBDE820404FF0000645
:100B80004FF000074FF000084FF0000B21F0070175
:100B9000AC46ACE8C009ACE8C009ACE8C009ACE8B8
:100BA000C0098D46704710B50446AFF3008020465B
:100BB000BDE81040FFF723BB4FF0013C50F8042B79
:100BC00051F8043B9A4221D1A2EB0C03934313EA60
:100BD000CC1317D150F8042B51F8043B9A4215D18D
:100BE000A2EB0C03934313EACC130BD150F8042B64
:100BF00051F8043B9A4209D1A2EB0C03934313EA48
:100C0000CC13DBD04FF00000704700BFD01A01BA00
:100C1000B1FA81F101F0180122FA01F0CB40C1F1E3
:100C20002001DBB2C0B2C01A2CFA01F3D11A9143F1
:100C300011EAC311E6D1704701491820ABBEFEE7A7
:100C40002600020070475FEA400C08BF91F0000FD9
:100C50004FEA8C234FEAC12243EA51514FEA1C501C
:100C600018BF00F5F0404FEA300018BF41F00041D6
:100C70005FEA6C5C00F02980BCF1FF3F08BF40F0E8
:100C800080407047130C06BF12044FF0100C4FF059
:100C9000000C130E04BF12020CF1080C130F04BF5A
:100CA00012010CF1040C930F04BF92000CF1020C22
:100CB000D30F04BF52000CF1010C11464FF000029B
:100CC000A0F11F00A0EB0C00704711F0004F08BF0F
:100CD000704731F000413FF4D5AF0B0C06BF09045B
:100CE0004FF0100C4FF0000C0B0E04BF09020CF17A
:100CF000080C0B0F04BF09010CF1040C8B0F04BF8F
:100D000089000CF1020CCB0F04BF49000CF1010C5F
:100D1000CCF12003A0EB0C0022FA03F302FA0CF250
:100D200041EA030100F10100704720F07F4C80EAA6
:100D3000030023F07F47ACEB070303F57C5300F07F
:100D4000004003F1FF032DE980494FEA154B09B438
:100D50004FEA144325EA0B4E24EA03480FF2042617
:100D600006EB132749083E785FEA320203FB066769
:100D7000C7F5000707FB06F64FEA54374FEAD64699
:100D800006F1020607FB066CCCF1005C4FEA1C473B
:100D90002CEA074C07FB06F40CFB06F504EB1546A2
:100DA0004FEA961634BF00204FF000404FEAD1378B
:100DB00006FB07FC4FEA1C4C0CFB0BF7D21B03FB9A
:100DC0000CF761EB07010CFB0EF7B0EB074072EB81
:100DD00017420CFB08F734BFA2EB0742B2EB074205
:100DE00061EB17414FEA0C444FEA910706FB07FC01
:100DF0004FEA1C4C0CFB0BF7B0EBC74072EB5732C1
:100E000003FB0CF734BFA2EBC742B2EBC74261EB66
:100E100057310CFB0EF7B0EBC70072EB57720CFBAF
:100E200008F734BFA2EBC702B2EBC70261EB577100
:100E3000039F4FEA816141EA921104EBCC044FEA2F
:100E4000D1374FEA826206FB07FC42EA90124FEA72
:100E500080604FEA1C4C0CFB0BF7D21B03FB0CF71A
:100E600061EB07010CFB0EF7B0EB074072EB17428A
:100E70000CFB08F734BFA2EB0742B2EB074261EB71
:100E800017414FEA8C554FEA910704EB9C2406FB6F
:100E900007FC4FEA1C4C0CFB0BF7B0EBC74072EBA6
:100EA000573203FB0CF734BFA2EBC742B2EBC74289
:100EB00061EB57310CFB0EF7B0EBC70072EB5772CA
:100EC0000CFB08F734BFA2EBC702B2EBC70261EB21
:100ED000577115EB4C254FEA816141EA92114FEAB7
:100EE00082624FEAD13742EA901206FB07FC44F1D6
:100EF00000044FEA80604FEA1C4C0CFB0BF7D21B3E
:100F000003FB0CF761EB07010CFB0EF7B0EB07409E
:100F100072EB17420CFB08F734BFA2EB0742B2EBAF
:100F2000074261EB174115EB1C154FEA813141EA8D
:100F300092414FEA823242EA90424FEA80304FEAD1
:100F40000C7644F1000448EA03434EEA0B484FF0A4
:100F5000000EB2EB080C71EB030724BF6246394662
:100F60004EEB0E0E4FF0000B0018524149414BEB77
:100F70000B0BB2EB080C71EB03077BF1000B24BFEA
:100F8000624639464EEB0E0E4FF0000B00185241F0
:100F900049414BEB0B0BB2EB080C71EB03077BF1F8
:100FA000000B24BF624639464EEB0E0E51EA020793
:100FB00018BF46F0010616EB0E7655F1000254F10B
:100FC000000103D5BDE88901BDE80088BDE88901BD
:100FD000BDE80048B619524141EB0101A3F10103FC
:100FE000704780807F7E7D7C7B7A79787776767596
:100FF0007473727171706F6E6E6D6C6C6B6A6A690E
:101000006868676666656464636362616160605FA7
:101010005F5E5E5D5D5C5C5B5B5A5A595958585720
:101020005756565555555454535352525251515088
:1010300050504F4F4F4E4E4D4D4D4C4C4C4B4B4BDB
:101040004A4A4A4949494848484747474746464621
:10105000454545444444444343434342424242415C
:101060004141002B9C4630D477002BD01CB54FEA71
:10107000370703B44FF010004FF01001BAF1000F22
:1010800006D0BCF1000FDCBF40F0080040F00801C2
:101090004FF000000FBCBDE810400BF1010BBBF19D
:1010A000010F08BF5FEA170722BF12F1010211F119
:1010B00001014FF0004143F1000300F0004043EA1A
:1010C00000007047F9D35708D0E746EA064613F107
:1010D000400F4FEA16461FDD13F1200FDFBF164306
:1010E0000A46002120335B42BED0C3F1200746EA06
:1010F000064602FA07F74FEA164646EA0706C3F124
:10110000200722FA03F201FA07F721FA03F14FF060
:10111000000342EA0702A7E746EA020646EA064655
:101120004FEA164646EA0106BCBF46EA0646360CBA
:101130004FF000034FF000024FF0000194E72DE95B
:10114000804C9A46934670B491E8380007C831EA5B
:10115000400C48BF34EA430C03D5FFF7E6FDFFF728
:1011600080FFF0BCBDE8008C2DE9804C9A46934688
:1011700070B491E8380007C810F0804F08BF13F032
:10118000804F03D100F005F8FFF76BFFF0BCBDE81E
:10119000008C20F07F4780EA030023F07F4C07EBB0
:1011A0000C03A3F57C5300F00040A3F1FE0392F082
:1011B000000F00F0B38095F0000F00F077802DE96C
:1011C00001494FEA11404FEA144621EA004800FB6A
:1011D00006FC24EA064708FB06F607FB08F800FBB6
:1011E00007F718EB06484CEB164C4FEA124B18EB7E
:1011F00007484FEA15464CEB174022EA0B4E0BFB13
:1012000006FC25EA06470EFB06F607FB0EFE0BFB67
:1012100007F71EEB064E4CEB164C4FF000061EEB8C
:10122000074E4CEB174B18EB0B0840F1000018EB86
:101230000E0B58EB000840F100008F1A4FF0000130
:101240003CBFC943661B14BFB5EB040C00213CBF77
:10125000C943F61B4FEA17444EEA8E0E27EA0445AF
:101260004FEA1C4704FB07622CEA074C05FB07F713
:101270000CFB05F604FB0CFC16EB074642EB174291
:1012800016EB0C4642EB1C421BEB060658EB020227
:10129000414146EA9E0601D5BDE80189B619524191
:1012A00041EB0101A3F10103BDE801894FEA1445B7
:1012B0004FEA114724EA054621EA074C05FB07F4EB
:1012C00006FB07F70CFB06F105FB0CFC11EB0741D5
:1012D00044EB17444FEA124711EB0C4144EB1C441A
:1012E00022EA074C05FB07F206FB07F70CFB06F6A4
:1012F00005FB0CFC16EB074642EB174216EB0C46BF
:1013000042EB1C456A1854F1000148BF7047B619FA
:10131000524141EB0101A3F10103704795F0000F29
:1013200037D04FEA11424FEA144721EA024624EA35
:10133000074C02FB07F106FB07F70CFB06F402FB68
:101340000CFC14EB074441EB17414FEA154714EB33
:101350000C4441EB1C4125EA074C02FB07F506FB58
:1013600007F70CFB06F602FB0CFC16EB074645EBF9
:10137000174516EB0C4645EB1C42121951F10001C2
:1013800048BF7047B619524141EB0101A3F1010377
:1013900070474FEA14454FEA114724EA054621EA0F
:1013A000074C05FB07F106FB07F70CFB06F24FF0B5
:1013B000000605FB0CFC12EB074241EB174112EB58
:1013C0000C4251EB1C4148BF7047921841EB0101A0
:1013D000A3F101037047000010B5084C0022102152
:1013E000204600F030FD022004F0B8FB2046012228
:1013F000BDE81040102100F026BD000000080140AB
:101400002DE9FF41A0200124CDE90004DFF84C8044
:10141000032569460395404600F014FC0122602133
:10142000404600F010FD40200026CDE90006694648
:101430000294404600F006FC10270097CDE90164B5
:101440006946074800F0FEFBCDE900746946404656
:10145000039500F0F7FBBDE8FF81000000080140A4
:101460000010014010B5084C00221021204600F069
:10147000EAFC082004F072FB20460122BDE810407F
:10148000102100F0E0BC000000080140FEE7000071
:10149000084900B5098981420AD0A0F57F41FF398A
:1014A00006D028B1B12803D002F066FD002000BDAF
:1014B000012000BD440100200348002181704163E8
:1014C000C1610162416270470C01002010B50F49F3
:1014D000052808D2DFE800F0030514161800812063
:1014E00000E091200870C020487000208870C8700B
:1014F000064A042104F05CFBBDE8104003F06EBF17
:10150000A120EFE7B120EDE70120EBE78400002008
:10151000014800F0FDB900003003002030B590F81C
:1015200040500124AC40C56B6C6004686360436844
:10153000102B036803D099600068C26030BD9A60C8
:101540000068C16030BD000010B5234890B000793C
:1015500000283ED0022837D2DFE800F036011F49CC
:1015600000230B6000F008F969461D4A04E0D41816
:10157000647ACC545B1CDBB28342F8D319499DF8E2
:101580000000086018499DF80100087017499DF88F
:10159000020008709DF8030015499DF8042002EB35
:1015A000002008609DF8050012499DF8062002EB16
:1015B000002008609DF807000F499DF8082002EB05
:1015C00000200860FFF778FF10B0BDE8104002F07F
:1015D000D3BC10B010BD0000440100202C0100203D
:1015E000F0030020100100200C0100200D0100205C
:1015F00014010020180100201C0100207047000089
:10160000F0B52A4C2A4D0126226942B12146022713
:101610004969491C012A0AD0022A39D114E0052857
:1016200004D10021616128702661E161F0BD616132
:1016300068540229FAD32761A878697800EB012061
:10164000E0613B2824D2F0BD61613B2920D268547F
:10165000E0698142F7D368790102A8790843FFF76E
:1016600017FFA8B1E879297A4FF2021301EB0020A5
:10167000C21A0421984216D006DC6FF4704140185B
:101680000AD0C02804D109E00F2A09D0102A0AD0B4
:10169000BDE8F04002F070BC2671F0BD2771F0BDCE
:1016A00003202071F0BD2171F0BD00004401002035
:1016B000F003002072B6074C4FF40065A614002218
:1016C0002946204600F0BFFB00223146204600F0AC
:1016D000BAFBF4E70008014070B50024FFF7F6FEFE
:1016E000FFF7C0FE4FF47A761B4D02E0641CB44253
:1016F00005D81021284600F0A1FB0028F6D103F000
:101700001DFE0446FFF768FE1448210206D501219C
:101710004170E04320F07F44641C01E000214170EF
:10172000204605F069FC0E4905F0AEFC05F096FA7E
:101730000C4A0D4B05F0AAF800220C4B04F04EFFAA
:1017400000220B4B04F0A2FE04F06EFEBDE87040D8
:10175000084905F023BB0000001001407C00002078
:1017600000007A44CBA145B6F3FD0340FEFF2F41B4
:1017700000C06240000020410448F5228178407892
:1017800002EB00200844C0B270470000F0030020C4
:1017900010B590F821100022022905D004218163A0
:1017A00080F82020012010BD01680B6823F00E0393
:1017B0000B6001680B6823F001030B6090F8403068
:1017C000C46B012101FA03F3636080F8211080F8F3
:1017D0002020104610BD00002DE9F05F90F8211088
:1017E0000024022903D004218163012485E00168DB
:1017F0000A6822F00E020A6001680A6822F00102FB
:101800000A603F4E3E4FB215DFF8F4C0DFF8F090AB
:10181000DFF8ECA0DFF8E8B0DFF8E4E00168783F3B
:1018200013011502ACF1640CA9F15009AAF13C0AAC
:10183000ABF1280BAEF1140E4FF48018B14227D94A
:10184000B9420ED0614512D049451DD0514518D03E
:10185000594518D0714501D1424615E0294EB14293
:1018600001D1012210E0274E1436B14201D11022DD
:101870000AE0244E2836B14206D0224A3C32914238
:1018800001D11A4600E02A461E49091F0A602BE0D2
:10189000B94213D0614517D0494522D051451DD0DA
:1018A00059451DD0714501D142461AE0B14202D1DD
:1018B0004FF0807215E0134EB14201D1012210E0C9
:1018C000104E1436B14201D110220AE00D4E2836D6
:1018D000B14206D00B4A3C32914201D11A4600E097
:1018E0002A46074980394A60012180F821100021E9
:1018F00080F82010416B01B188472046BDE8F09F79
:10190000800002400804024090F821007047000067
:101910002DE9F05FC16B0A6801680B68046C4FF039
:10192000040808FA04F8844D844E854FDFF814C289
:10193000DFF81492DFF814A2DFF814B2DFF814E233
:1019400018EA020F65D05FEA437862D50A6892060A
:1019500003D40A6822F004020A60DFF8F0814FF431
:101960008062016808F1140813011402414524D96A
:10197000A9420DD0B1420FD0B9421AD0614515D05D
:10198000494515D0514501D1120312E0594501D105
:1019900004220EE0714501D140220AE06D4D14355C
:1019A000A94206D06B4A2832914201D11A4600E082
:1019B00022466749091F0A6029E0A94213D0B142B3
:1019C00015D0B94220D061451BD049451BD05145A7
:1019D00002D14FF4800217E0414502D14FF08062FE
:1019E00012E0594501D104220EE0714501D1402297
:1019F0000AE0584D1435A94206D0564A2832914281
:101A000001D11A4600E022464B4908394A60C16AB2
:101A100071E04FF0020808FA04F818EA020F70D0DB
:101A20005FEA83786DD50A68920606D40A6822F0C8
:101A30000A020A60012180F82110DFF810814FF4BA
:101A40000072016808F1140813011402414524D9F9
:101A5000A9420DD0B1420FD0B9421AD0614515D07C
:101A6000494515D0514501D1120312E0594501D124
:101A700002220EE0714501D120220AE0354D1435D5
:101A8000A94206D0334A2832914201D11A4600E0D9
:101A900022462F49091F0A6029E0A94213D0B1420A
:101AA00015D0B94220D061451BD049451BD05145C6
:101AB00002D14FF4001217E0414502D14FF00072FD
:101AC00012E0594501D102220EE0714501D12022D8
:101AD0000AE0204D1435A94206D01E4A2832914210
:101AE00001D11A4600E02246134908394A60002114
:101AF00080F82010816A00291CD0BDE8F05F0847FB
:101B0000FFE70825A540154214D01A0712D50A6828
:101B100022F00E020A6090F84020C36B012101FA06
:101B200002F25A60816380F82110002180F82010B1
:101B3000016BE0E7BDE8F09F080002401C00024096
:101B40003000024044000240580002406C00024055
:101B5000080402401C04024030B560B11A4B026810
:101B600014219A4209D2194B1344B3FBF1F18900B5
:101B7000016417490AE0012030BD134B5B42134456
:101B8000B3FBF1F1890001640F490839C1630221F7
:101B900080F82110136843F6F0718B43F0E90114CB
:101BA0002143D0E902452C43214304692143446980
:101BB00021438469214319431160002141630122BB
:101BC00042770177084630BD08040240F8FFFDBFA8
:101BD0000000024070B5044690F82000002501285E
:101BE0000CD0012084F8200094F821600020012E00
:101BF00006D084F820000225284670BD022070BD62
:101C0000022684F82160A0632068066826F0010699
:101C100006602046FFF782FCE06A00282068016821
:101C200002D041F00E0106E021F0040101602068BD
:101C3000016841F00A0101602068016841F001017A
:101C40000160D9E72DE9F84FDFF8C8910024A9F128
:101C5000040B23460F2709F1040AABF1040ED1E06F
:101C60000125A54006EA0502AA4276D1DFF8A8C1FF
:101C70004E68A6EB0C0866452BD00DDC032E34D045
:101C800005DC36B3012E19D0022E2FD11BE0112E08
:101C900016D0122E2AD119E0B8F5881F19D006DC0B
:101CA000B8F5803F15D0B8F5801F1FD111E0B8F509
:101CB000001F0ED0B8F5041F18D10AE0CB6815E05C
:101CC000CB681B1D12E0CB6808330FE0CB680C33E8
:101CD0000CE08B682BB1012B4FF0080303D045615A
:101CE00004E0042302E0056100E00023FF2A01D89C
:101CF000064601E000F104064FEA840501D9A5F18A
:101D00002005D6F8008007FA05FC28EA0C0803FA3B
:101D100005F548EA0508C6F800804D68ED0070D565
:101D20003E4DAE6946F00106AE61AD6924F0030692
:101D300005F0010500953A4D06EB050CDCF808505E
:101D4000A607360F07FA06F825EA0805DFF8D4805B
:101D5000404503D14FF0000825E052E0DFF8C8808D
:101D6000404502D14FF001081DE0DFF8C08040453A
:101D700002D14FF0020816E0DFF8B480404502D1EE
:101D80004FF003080FE0DFF8AC80404502D14FF080
:101D9000040808E0DFF8A080404502D14FF00508B4
:101DA00001E04FF0060808FA06F848EA0508CCF802
:101DB00008804D68D9F80060ED024D4601D5164304
:101DC00000E096432E604D68DAF80060AD0255469B
:101DD00001D5164300E096432E604D68DBF80060A5
:101DE000AD035D4601D5164300E096432E604D6875
:101DF000DEF80060ED03754601D5164300E096431A
:101E00002E60641C0A681646E2407FF429AFBDE8E4
:101E1000F88F00000804014000001110001002407B
:101E20000000014000080140000C0140001001408A
:101E30000014014000180140001C01408068084067
:101E400000D0012070470AB1016170470904FBE727
:101E500001488068704700004400002070477047C8
:101E60002DE9F041016804464A694E6890F83E0049
:101E70000025D743FA050BD4F243D20508D46FF4FA
:101E8000807201254A6121680A6842F400420A60B2
:101E9000B90508D4F143C90505D422686FF400716F
:101EA00045F002055161790525D4F143C90522D4D5
:101EB000638D94F83D10226B202808D13BB921296D
:101EC00010D029290ED0282901D1212A0AD0226830
:101ED0006FF48061516145F00405102806D0402858
:101EE00004D008E0204601F051FF04E020680168BA
:101EF00041F400710160380508D4F043C00505D4F1
:101F000021686FF4006045F008054861002D07D096
:101F1000206C284320642046BDE8F04101F0A4BBBA
:101F2000BDE8F0812DE9F047026800215368C66AD8
:101F300090F83E4090F83D50102C12D0402C10D01C
:101F4000046C002C7DD05469E443A6077AD4DE43A8
:101F5000B60577D4036C03B19169BDE8F04701F091
:101F6000F1BE976951694FF42A0CC9435FEAC17801
:101F70004FF02A4904D066452AD04E4528D010E0BB
:101F8000DE43B6050DD4C16A614501D1012103E0EC
:101F9000C16A494501D10821C162BDE8F04701F09D
:101FA00037BE0E0716D4DE43B60513D4416CC9B252
:101FB0001161416B09B1896A29B9816B002907D088
:101FC000896A002904D00068416841F400614160D9
:101FD000BDE8F0878E0706D4DE43B60503D4BDE81E
:101FE000F04701F069BDFE43526876074FEA02529E
:101FF0001DD4002AECDB0A0608D4DA43520505D4C6
:10200000490705D5BDE8F04701F0FABC4907DFD420
:10201000D9438905DCD4212D05D0402CD8D1BDE889
:10202000F04701F03BBEBDE8F04701F0A7BC002A35
:10203000CEDB4A060BD4DA43520508D4490708D54B
:1020400001E00DE00EE0BDE8F04701F023BC4907D8
:10205000BED4D9438905BBD4BDE8F04701F0B0BB7D
:10206000916970E7E10606D4D943890503D4BDE838
:10207000F04701F0D3BE2821212D27D0292D25D0CE
:10208000650655D4DD436D0552D4640752D590F8EA
:102090003D30448D002C9BD01269446A2270426A04
:1020A000521C4262428D521E4285428D002A8FD1BF
:1020B0002A2B8DD10268536823F480635360222257
:1020C000026380F83D1000F057F981E7250623D41C
:1020D000DD436D0520D4640720D590F83D30448D54
:1020E000002CF2D0446A24781461426A521C426285
:1020F000428D521E4285428D002AE6D1292BE4D121
:102100000268536823F4806353602122026380F8DD
:102110003D1000F032F95BE76107D6D4D943890559
:10212000D3D4418D0029D0D0416A097811610AE0E9
:102130006107CAD4D9438905C7D4418D0029C4D0C9
:102140001169426A1170416A491C4162418D491E00
:1021500041853DE77047000070B5040025D094F834
:102160003D00002520B984F83C50204600F0BEF820
:10217000242084F83D002068016821F001010160FD
:102180002068016841F4004101602068016821F481
:102190000041016000F020FA4D4A6168914201D887
:1021A0004C4900E04C49884201D2012070BD4B49A6
:1021B0002368B0FBF1F15E6826F03F060E435E60D7
:1021C0006368934206D94FF4967359434FF47A7378
:1021D000B1FBF3F12368491C1E6A26F03F06314328
:1021E00019626168914210D84900401EB0FBF1F2BB
:1021F000521CC2F30B02042A01D2042022E0B0FBDD
:10220000F1F0401CC0F30B001CE0A268F2B301EB3C
:10221000C10303EB0116431EB3FBF6F35B1C43F44F
:1022200080431B0549D092B301EBC10202EB0111BF
:10223000401EB0FBF1F0401CC0F30B0040F48040A6
:1022400040F400402168CA694CF6FF739A4310437A
:10225000C861D4E9071001432068026822F0C00277
:1022600011430160D4E9030101432068826848F208
:10227000FF339A4311438160D4E905010843216883
:10228000CA6822F0FF021043C86001E00EE016E0C9
:102290002068016841F0010101602564202084F874
:1022A0003D00256384F83E50002070BD01EB4106DF
:1022B000431EB3FBF6F35B1CB3E70120C2E701EB5F
:1022C0004101401EB0FBF1F0401CC0F30B00B7E72A
:1022D000A086010080841E0000093D0040420F00DE
:1022E00070477047704770477047000010B586B060
:1022F0000021009101910291039100681A498842DE
:1023000030D11A4CA06940F00800A061A06969466C
:1023100000F008000490C0200090122001900320DB
:1023200003901348FFF78EFCE06940F40010E06171
:10233000E069002200F40010049011461F2000F014
:1023400083F81F2000F072F800221146202000F0D0
:102350007BF8202000F06AF806480068416841F4E4
:10236000E061416006B010BD005400400010024022
:10237000000C0140640100207047704702488168EA
:10238000027811448160704744000020074810B56E
:10239000016841F010010160032000F075F8002091
:1023A00000F006F800F024F8002010BD00200240E4
:1023B00070B50D4D04464FF47A712878B1FBF0F0FA
:1023C0000A490968B1FBF0F000F0F2FB48B9102CA3
:1023D00007D200222146501E00F036F800206C6023
:1023E00070BD012070BD000044000020500000209E
:1023F0000C4808B5816941F001018161816901F0F2
:1024000001010091C16941F08051C161C06900F0D2
:10241000805000900448416821F0E06141F0007173
:10242000416008BD0010024000000140002809DBA7
:1024300000F01F02012191404009800000F1E020DE
:10244000C0F8001170470000F0B40E4B1B680C463A
:10245000C3F30223C3F10705042D00D90425191D78
:10246000072901D2002300E0DB1E012606FA05F150
:10247000491E214099409E40761E16403143F0BCD3
:1024800003F03ABC0CED00E0064900F007020868D2
:102490004FF6FF03184040EA0220034A1043086049
:1024A000704700000CED00E00000FA052DE9F04750
:1024B0000F46050061D0434E306800F00700B84277
:1024C00009D2306820F0070038433060306800F0EF
:1024D0000700B84251D128683B4C810712D540070C
:1024E00003D5606840F4E06060602878000703D599
:1024F000606840F4605060606068A96820F0F00097
:10250000084360602878C00728D06868012810D088
:102510002168022810D0890700292EDA616821F08D
:10252000030101436160FFF793FC804641F2883963
:102530000DE021688903EFE78901EDE7FFF788FCEB
:10254000A0EB0801494502D90320BDE8F087606887
:10255000696800F00C00B0EB810FEFD1306800F03B
:102560000700B8420BD9306820F0070038433060CC
:10257000306800F00700B84201D00120E5E7287874
:10258000400705D56068E96820F4E06008436060B2
:102590002878000706D56068296920F4605040EA71
:1025A000C100606000F038F86168084AC1F30311A7
:1025B000515CC8400649086006480068FFF7F8FE0D
:1025C0000020C2E7002002400010024064740008AE
:1025D0005000002048000020044805490068496870
:1025E000044AC1F30221515CC840704750000020EA
:1025F00000100240747400080448054900684968E6
:10260000044AC1F3C221515CC84070475000002009
:1026100000100240747400080E4A51680E4801F020
:102620000C03042B11D0082B0FD10C48C1F38343AA
:10263000C903C05C0AD55168084AC1F34041921EE3
:10264000515C054A5043B0FBF1F0704704494843E0
:10265000704700000010024000127A005474000815
:1026600000093D002DE9F84F040070D02078C04DDE
:10267000C00749D06868C0F38100012807D06868A6
:10268000C0F38100022809D16868C00306D5286814
:10269000800339D560680028E7D035E06068B0F580
:1026A000803F0BD010B1B0F5A02F11D0286820F4D6
:1026B00080302860286820F4802002E0286840F4F8
:1026C00080302860606890B1FFF7C2FB06460AE0E0
:1026D000286840F480202860F0E700BFFFF7B8FBCF
:1026E000801B642873D828688003F7D50CE0FFF7B7
:1026F000AFFB064605E000BFFFF7AAFB801B64287E
:10270000F0D828688003F7D420789A4E80074FF0DD
:1027100001094FF0000839D5686810F00C0F07D098
:102720006868C0F38100022809D16868C00306D434
:102730002868800714D52069012808D110E0206995
:10274000B0B1C6F80090FFF783FB074605E00AE149
:10275000FFF77EFBC01B0228C4D828688007F7D586
:102760002868616920F0F80040EAC10028600DE0A7
:10277000C6F80080FFF76CFB074604E0FFF768FB34
:10278000C01B022823D828688007F7D420780007C8
:102790002CD57948A169D9B1C0F80090FFF758FB52
:1027A000074604E0FFF754FBC01B02280FD8686AF5
:1027B0008007F7D571484FF4FA510068B0FBF1F08B
:1027C000009000BF0098411E0091FAD20EE080E018
:1027D000C0F80080FFF73CFB074604E0FFF738FB3A
:1027E000C01B022875D8686A8007F7D42078400794
:1027F00060D5E8690027C00008D4E86940F080503F
:10280000E861E869012700F0805000905C480168A9
:10281000C90513D40168834641F480710160FFF754
:1028200017FB824606E000BFFFF712FBA0EB0A0091
:1028300064284ED8DBF80000C005F5D5E068012813
:102840000AD008B1052813D0286A20F001002862B8
:10285000286A20F0040002E0286A40F001002862A3
:10286000E06841F2883B98B1FFF7F2FA82460BE04C
:10287000286A40F004002862EEE700BFFFF7E8FA9C
:10288000A0EB0A0159455AD8286A8007F6D50CE012
:10289000FFF7DEFA824605E0FFF7DAFAA0EB0A015D
:1028A00059454CD8286A8007F6D41FB1E86920F052
:1028B0008050E861E06988B36968C1F38101022949
:1028C00044D00228C6F8608004D0FFF7C1FA04465D
:1028D00038E034E0FFF7BCFA074604E0FFF7B8FA47
:1028E000C01B02282BD828688001F7D4206AB0F5D5
:1028F000803F05D16868A16820F400300843686013
:10290000D4E908010843696821F474110843686038
:10291000C6F86090FFF79CFA044606E025E000BF89
:10292000FFF796FA001B022809D828688001F7D51E
:102930001BE000BFFFF78CFA001B022802D903201E
:10294000BDE8F88F28688001F4D40EE00128F7D0A4
:102950006868226A00F48031914204D1616A00F40F
:102960007010884201D00120EAE70020E8E700006B
:102970000010024000004242800442425000002009
:10298000007000407047000038B504460068426897
:102990008168C9434B0606D5CB0704D1D3435B06F8
:1029A00001D4216C05E08B0708D4D3431B0605D462
:1029B000616C01B02046BDE8304008478B0601D568
:1029C0004B0646D4D3439B0643D44B060AD494F813
:1029D0005130032B3ED0636D43F004036365C3683D
:1029E00083680093890609D4616D41F00101616536
:1029F00081680091016821F040010160606D00284C
:102A000027D02068416821F0E0014160012084F86E
:102A10005100900722D02068416821F003014160F5
:102A2000104DE06C40B14563E06CFEF7D5FE18B187
:102A3000606D40F040006065A06C002809D04563DF
:102A4000A06CFEF7C9FE002803D0606D40F0400086
:102A5000606538BDC1688068009038BD2046FFF7CA
:102A600091FF38BD2154000870B5040009D0606A98
:102A7000002540B125616561A56294F8510040B11F
:102A80000CE0012070BD6068B0F5827FF4D0E56194
:102A9000F2E784F85050204600F040F8022084F815
:102AA00051002068016821F040010160A08821895F
:102AB00000F4827001F404410843A18901F400612B
:102AC0000843217C01F002010843217D01F001014E
:102AD0000843218B01F400710843217F01F0380184
:102AE000084394F8201001F080010843218D01F47F
:102AF0000051084321680860A069042101EA1040E0
:102B0000216848602068C16921F40061C161656580
:102B1000012084F85100002070BD000030B585B060
:102B20000024009401940294039400681C49884294
:102B300033D11C48C16941F48041C161C16901F4CC
:102B400080410491816941F0080181618069164DDD
:102B500000F0080004904FF4204000900220019003
:102B60000320039069462846FFF76CF84FF4804035
:102B7000CDE90004694628460294FFF763F8002275
:102B800011462420FFF760FC2420FFF74FFC074884
:102B90000068416841F0A001416005B030BD00000F
:102BA0000038004000100240000C0140B801002035
:102BB00010B5401EB0F1807F01D3012010BD4FF051
:102BC000E02460610F21601703F096F80020A061F7
:102BD00007202061002010BD7047704770B590F845
:102BE0003C20012A2CD0012480F83C40022280F8AD
:102BF0003D2003685A689D6822F070060A683243D7
:102C00005A60104B02689A420ED00F4B9A420BD07A
:102C1000B2F1804F08D00D4B9A4205D00C4B9A422E
:102C200002D00C4B9A4204D1496825F08003194325
:102C3000916080F83D40002180F83C10084670BD4E
:102C4000022070BD002C014000340140000400400F
:102C500000080040000C004010B5040003D094F8B8
:102C60003D0010B107E0012010BD002084F83C00B9
:102C7000204600F01FF8022084F83D00211D206846
:102C800002F046FC012084F8460084F83E0084F8F7
:102C90003F0084F8400084F8410084F8420084F842
:102CA000430084F8440084F8450084F83D00002087
:102CB00010BD000008B500680B49884212D10B48CE
:102CC000816941F4006181618069002200F4006043
:102CD000009011461920FFF7B7FBBDE80840192006
:102CE000FFF7A4BB08BD0000002C0140001002400B
:102CF00090F83D10012901D001207047022180F891
:102D00003D100168CA6842F00102CA6000680E49BD
:102D100088420ED00D4988420BD0B0F1804F08D0C8
:102D20000B49884205D00B49884202D00A498842A3
:102D300004D1816801F00701062903D0016841F040
:102D40000101016000207047002C01400034014067
:102D50000004004000080040000C004070B504462C
:102D600090F83C000025012817D0012684F83C602B
:102D7000022084F83D002068826822F0770222F465
:102D80007F4282600868502838D00DDC20284FD060
:102D900005DC90B3102811D14AE0022070BD302824
:102DA00046D040280AD13BE060282FD070280DD0B3
:102DB000B0F5805F03D0B0F5005F12D0012584F834
:102DC0003D60002084F83C00284670BDCB68D1E906
:102DD0000121206802F0E2FB2068816841F0770160
:102DE00009E0CB68D1E90121206802F0D7FB206817
:102DF000816841F480418160E1E719E0CA6849686F
:102E0000206802F0DDFB5021206806E0CA684968AE
:102E1000206802F0E6FB6021206802F0C9FBCEE7E3
:102E2000CA684968206802F0CBFB40212068F4E7BB
:102E3000226801461046F0E7704770B50446006806
:102E400001694FF00005C943890715D4C168C9431A
:102E5000890711D4E91E016101202077206880696B
:102E60008007204602D0FFF7E7FF04E000F098F863
:102E7000204600F096F8257720680169C943490784
:102E800017D4C168C943490713D46FF00401016125
:102E9000022020772068806910F4407F204602D00D
:102EA000FFF7CAFF04E000F07BF8204600F079F855
:102EB000257720680169C943090716D4C168C94349
:102EC000090712D46FF008010161042020772068FF
:102ED000C0698007204602D0FFF7AEFF04E000F093
:102EE0005FF8204600F05DF8257720680169C94346
:102EF000C90617D4C168C943C90613D46FF01001BD
:102F00000161082020772068C06910F4407F2046C6
:102F100002D0FFF791FF04E000F042F8204600F0F5
:102F200040F8257720680169C943C90708D1C168FD
:102F3000C943C90704D1891E0161204600F032F857
:102F400020680169C943090609D4C168C943090653
:102F500005D46FF0800101612046FFF73DFE206837
:102F60000169C943490609D4C168C943490605D462
:102F70006FF040010161204600F082F8206801698D
:102F8000C94389060BD4C168C943890607D46FF0C9
:102F9000200101612046BDE87040FFF71EBE70BDF4
:102FA00070477047344930B4884263D13348416830
:102FB000012901DA012200E00022491C4A430121D3
:102FC0004260012A00D18160C368052B01DA012229
:102FD00000E000225B1C5A43C260052A00D1016157
:102FE00042690A2A01DA012300E00023521C5343FC
:102FF00043610A2B00D18161C269642A01DA01238D
:1030000000E00023521C5343C361642B00D10162D2
:10301000436A4FF4FA74A34201DA012200E000226D
:103020005B1C5A434262A24200D18162C26A4FF4E1
:103030007A74A24201DA012300E00023521C5343B8
:10304000C362A34200D10163416B41F288339942CC
:1030500001DA012200E00022491C4A4342639A42FD
:1030600003D1816B21B10021816330BC00F09ABF94
:103070000121F9E730BC7047100200200000002059
:10308000704738B5044690F84200202801D002204D
:1030900038BD61B15AB10120206300206063204631
:1030A00002F0E2FC0028F3D1216B012901D00120BC
:1030B00038BD21680A684968009121680C3151E8DF
:1030C000002F42F0100241E80023002BF5D138BD5B
:1030D00070477047F8B5016804460868CA684B69CC
:1030E00010F00F0F4FF0000559D003F0010602F465
:1030F0009077374365D0C10705D0D10503D5616C02
:1031000041F001016164410705D5D90703D0616C25
:1031100041F002016164810705D5D90703D0616CD4
:1031200041F004016164010707D502F02001314339
:1031300003D0616C41F008016164616C00293AD0F0
:10314000800604D5900602D5204602F0CFFB206809
:103150004069616CC0F38010090700D460B3204659
:1031600002F08FFB20684069400621D520681430AA
:1031700050E8001F21F0400140E80012002AF5D17C
:10318000E06BA8B16D494163E06BFEF725FB0028B9
:1031900011D0E06B416B01B0BDE8F04008478306F9
:1031A0000FD593060DD52046BDE8F84002F09EBB32
:1031B0002046FFF78EFFF8BD2046FFF78AFF6564C3
:1031C000F8BD266B2023012E7CD1C6067AD5D60603
:1031D00078D508684868009048694FF002064006B4
:1031E00040D5E16B086840680004000CE8D0A28D6F
:1031F0008242E5D9E085886920282DD020680C30EE
:1032000050E8001F21F4807140E80012002AF5D137
:103210002068143050E8001F21F0010140E800123E
:10322000002AF5D12068143050E8001F21F0400139
:1032300040E80012002AF5D184F842302563206866
:103240000C3050E8001F21F0100140E80012002A65
:10325000F5D1E06BFEF79CFA6663A08DE18D401A14
:1032600081B22AE0A08DE18D401A81B2E08D002864
:10327000A6D00029A4D022680C3252E8000F20F416
:10328000907042E80007002FF5D12068143050E814
:10329000002F22F0010240E80027002FF5D184F82A
:1032A0004230256320680C3050E8002F22F01002D5
:1032B00040E80023002BF5D166632046FFF708FFA6
:1032C000F8BDFFE705062BD5150629D594F8410072
:1032D0002128F5D1A068B0F5805F01D12069B0B197
:1032E000206A411C2162216800784860E08C401E01
:1032F0000004000CE084E3D12068C16821F0800163
:10330000C1602068C16841F04001C160D8E7206A0F
:103310000088C0F308004860206A801C2062E5E74E
:103320004006CDD55006CBD5CA68204622F04002D3
:10333000CA6084F8413000F015F9C1E785570008EC
:1033400070B5040004D094F84100002510B106E0E7
:10335000012070BD84F84050204600F023F824205E
:1033600084F841002068C16821F40051C160204602
:1033700002F01EFB2068016921F490410161206880
:10338000416921F02A0141612068C16841F400517E
:10339000C1606564202084F8410084F842006563C0
:1033A000002070BDF0B585B0002400940194029413
:1033B0000394054603685648DFF850C102210322F2
:1033C000544E0715634528D1836943F480438361D4
:1033D000836903F480430493836943F004038361A6
:1033E0008069039200F0040004900802CDE9000116
:1033F00069463046FEF726FCCDE900746946304642
:103400000294FEF71FFC002211462520FFF71CF84E
:103410002520FFF70BF8404842E0DFF800C1634584
:1034200045D1C36943F40033C361C36903F4003376
:103430000493836943F0040383618069039200F07D
:10344000040004900420CDE9000169463046FEF7EF
:10345000F9FB0820CDE90004694630460294FEF7E6
:10346000F1FB2D4E2E48D836C6E900048020C6E96F
:10347000024020203461C6E905403046F461FEF781
:103480006BFB08B1FEF716F9EE6300221146262009
:103490007562FEF7D9FF2620FEF7C8FF1E484830A8
:1034A0000068C16841F06001C16005B0F0BD1D4D0C
:1034B000AB42FAD1C36943F48023C361C36903F407
:1034C00080230493836943F0080383618069CDE915
:1034D000007100F00800CDE90320134D694628462D
:1034E000FEF7B0FBE814CDE90004694628460294D3
:1034F000FEF7A8FB002211462720FEF7A5FF272094
:10350000FEF794FF04489030CAE7000000380140FD
:103510000010024000080140580200200044004012
:103520006C00024000480040000C014070477047AA
:1035300090F84130202B01D00220704779B172B150
:1035400001628284C28400214164212180F84110FB
:103550000068C16841F08001C1600020704701200F
:103560007047000000680449884204D1002202210B
:103570000248FEF768BC7047004400400008014064
:10358000FEE700000148FEF76BBC0000640100206C
:103590000148FEF7C7BC00006401002038B5406A4E
:1035A000002190F83D202B4B46F2A8141B68B3FB7A
:1035B000F4F3C3EBC30303EB830300933BB15B1E44
:1035C000009303681B689B0505D5009BF6E7036C19
:1035D00043F020030364436B03B19962836B03B12F
:1035E000996203681C6824F480641C604185436B05
:1035F00003B15963836B03B1596303681C6824F0FA
:1036000001041C6090F83D402023602C0BD028243E
:1036100034EA02020FD080F83D3080F83E1000BF3F
:10362000FEF798FD38BD80F83D3080F83E1001640B
:10363000FEF714FC38BD0268136843F00103136001
:103640000268136843F480631360016380F83D40AF
:10365000E6E700005000002000684169C943090600
:1036600001D400210161704770B5044690F83D0017
:1036700094F83E10102901D0402906D1222804D107
:1036800021680A6822F400620A60282131EA0002F7
:103690004FF000054FF0200626D021684968090543
:1036A00005D4602803D084F83D6084F83E5025633B
:1036B00020684168090537D5416821F400614160FF
:1036C000606B90F821203C49012A11D04163606B66
:1036D000FEF782F838B32068016821F0010101602B
:1036E00084F83D60606B1CE0256384F83D10DFE7E3
:1036F000A06B4163A06BFEF76FF8A0B12068416931
:10370000C943490605D40069616A0870606A401CB3
:1037100060622068016821F00101016084F83D6069
:10372000A06B416B884710E094F83D10602910D0E1
:103730004169C943490605D40069616A0870606A35
:10374000401C60622046FEF705FD206CC1071CD1BD
:1037500015E084F83D6025644169C943490605D4F4
:103760000069616A0870606A401C606220680168D4
:1037700021F0010101602046FEF770FBE5E78107BB
:1037800003D4410701D4000704D52068416821F41F
:10379000E061416094F83D00216C49070BD5282871
:1037A00009D10648E062256384F83D6084F83E5004
:1037B0002046FEF795FD70BD9D3500080000FFFF17
:1037C00010B5C26A438D0168042B06D0438D032BCC
:1037D00008D0438D022B1DD012E04A6822F480628B
:1037E0004A600CE04B6823F480634B60042A06D0E7
:1037F000022A04D001680A6822F480620A60016823
:103800000969426A1170416A491C4162418D491E31
:10381000418510BD012A30D0102A2ED0042A30D084
:10382000022A2ED00A6842F400720A60016809690F
:10383000426A1170416A491C4162428D521E4285A2
:10384000026812690A70416A491C4162418D491E31
:10385000418501684A6822F440724A60202180F85C
:103860003D1090F83E200021402A80F83E100CD0F8
:1038700012210163FEF735FD10BD0A6822F4806253
:10388000D3E70A6842F48062CFE70163FEF72BFDBD
:1038900010BD000038B590F83D1022290FD1418DA0
:1038A00003290DD901680969426A1170416A491CEE
:1038B0004162418D491E4185418D032906D038BDA5
:1038C000C26A022A02D0012906D029B100684168E3
:1038D00021F48061416038BD274946F2A8130022D7
:1038E0000968B1FBF3F101EB81010091016820232C
:1038F000009C641E009422D00C68A405F8D40C68C7
:1039000024F480640C6001684C6824F4E0644C602A
:1039100001680969446A2170416A491C4162418D0C
:10392000491E418580F83D3090F83E1080F83E20D9
:1039300040291DD012210163FEF7D3FC38BD046C71
:1039400044F0200404644C6824F4E0644C60016892
:103950000969446A2170416A491C4162418D491ECE
:10396000418580F83D3080F83E20FEF7F3FB38BDFE
:103970000263FEF7B8FC38BD5000002010B5C26AE3
:1039800090F83D1021290BD1418D51B1416A026857
:1039900009781161416A491C4162418D491E418586
:1039A00010BD20230021082A13D0202A11D012F59F
:1039B000803F0ED00268546824F4E0645460112201
:1039C000026380F83E1080F83D3000BFFEF78AFCAD
:1039D00010BD0268546824F4E064546002681468FE
:1039E00044F400741460016380F83D3090F83E2088
:1039F00080F83E10402AE9D1FEF776FC10BD0000A9
:103A000010B590F83D1090F83E30C26A048DB4B104
:103A1000212903D0402B11D122290FD1418DE1B3AF
:103A200090F83E10402942D0416A0268097811613D
:103A3000416A491C4162418D491E418510BD2129C1
:103A4000E8D120230021082A13D0202A11D012F512
:103A5000803F0ED00268546824F4E0645460112260
:103A6000026380F83E1080F83D3000BFFEF73AFC5C
:103A700010BD0268546824F4E0645460026814685D
:103A800044F400741460016380F83D3090F83E20E7
:103A900080F83E10402AE9D100E002E0FEF724FC65
:103AA00010BD0068416821F48061416010BDBDE82F
:103AB000104000F0F3B8000078B590F83E50C26AAC
:103AC000046B90F83D6000230168222E73D1066DCF
:103AD0000EB9402D6FD0056D1DB90569B5F5404F84
:103AE0001BD0458D95B3468D484D012E20D0448D79
:103AF000022C4DD00C6844F480640C6001684C6862
:103B0000240579D5AA4273D0012A71D0082A6FD032
:103B1000102A6DD0202A6BD06EE04A698A69009223
:103B20000A6842F480720A60016D491C016578BD23
:103B3000AA4214D10A6822F480620A6001684A68C5
:103B4000120504D50A6822F4806217E0FFE74A698B
:103B50008A6900920A6842F400720A6050E0082AFA
:103B600010D0202A0ED0122C0AD0042A03D0022A08
:103B700001D0102AE6D10A6842F480620A603BE074
:103B8000012ADFD00A6822F480620A600168DEE759
:103B9000042A11D0022A0FD0102A0DD00C6844F448
:103BA00000640C6001684C698C6900940C6824F412
:103BB00080640C6008E025E00C6844F480640C60CC
:103BC00001684C698969009101684C68240517D522
:103BD000AA4207D0012A05D0082A03D0102A01D012
:103BE000202A0DD14A6842F480524A6008E0FFE77B
:103BF0004A6842F480524A6001684A6989690091C2
:103C0000036578BD48698869009078BD0000FFFFB2
:103C100090F83E10402910D00169B1F5804F19D0BD
:103C2000016DA9B3016D012910D1416C5FF0F10262
:103C300001F4407142EAD11106E0016D0029416CA6
:103C400005D0C9B241F0010100680161704701F07F
:103C5000FE01F9E790F83D102129416C09D0C9B265
:103C600041F0010102681161416B29B1896A49B9CA
:103C700002E001F0FE01F5E7816B0029E6D0896AD8
:103C80000029E3D00068416841F400614160704759
:103C9000FFE7416CF02201F44071CBE710B590F8DA
:103CA0003D10026D4AB1026D012A14D0026D022A44
:103CB00016D0BDE81040FFF7CFBCC16C0129816C64
:103CC00002D0C1F3072108E00268C9B21161016D99
:103CD000891C016510BD816CC9B20268116123E0C5
:103CE00022291CD0428D0AB1212920D0428D002AE0
:103CF000F0D12129EED101684A6822F4E0624A60DD
:103D000001680A6842F400720A60002101632022FF
:103D100080F83D2080F83E10FEF7E6FA10BD0168FD
:103D20000A6842F480720A60016D491CD1E7416A59
:103D3000026809781161416A491C4162418D491E3E
:103D4000418510BD38B50C4690F83D20002128254E
:103D5000954302680B4605D051699169009180F83E
:103D60003C3038BD556825F480655560E243540702
:103D700000D50121120601D5828900E0028B80F86E
:103D80003C3092B2FEF76BF838BD00002DE9F041EF
:103D900090F83D300446C26A002120261E4F00687C
:103DA0006FF48065082A01D0202A01D1282B04D085
:103DB000212B17D04561BDE8F081E762426822F40B
:103DC000E0624260206845612068026822F48062F7
:103DD0000260216384F83D6084F83E102046FEF7BF
:103DE0007FFAE8E7E7622122226384F83D6084F8E5
:103DF0003E10416821F4E06141602068456120681F
:103E0000016821F4806101602046FFF725FC20460F
:103E1000FEF7B3FACFE700000000FFFFF8B590F817
:103E20003D6004460068416821F4E061416020681B
:103E3000002541690091016841F00101016020689D
:103E4000016821F48061016020684168090520D57E
:103E5000474F222E48D02A2E46D0616B0968496808
:103E60006185618D19B1216C41F0040121644168C3
:103E700021F400614160606BFDF746FD012808D028
:103E8000606B4763606BFDF7A7FC10B1606B416B23
:103E90008847608D08B320684169C943490708D441
:103EA0000069616A0870606A401C6062608D401E33
:103EB000608520684169C943490608D40069616A80
:103EC0000870606A401C6062608D401E6085608D75
:103ED00018B1206C40F004002064206C00B3204630
:103EE000BDE8F840FFF7C0BBA16B09684968618570
:103EF000618D19B1216C41F004012164416821F404
:103F000000614160A06BFDF7FFFC0128C1D0A06BF0
:103F10004763A06BFDF760FC0028BAD0A06BB6E742
:103F20002A2E06D12563282084F83D002046FEF77E
:103F300023FA94F83D10202028290DD0216B222946
:103F400001D0222E07D1256384F83D0084F83E502D
:103F50002046FEF711FAF8BD0649E162256384F8B0
:103F60003D0084F83E502046FEF7BAF9F8BD000047
:103F70009D3500080000FFFF08490020084B08712C
:103F800048610861C86148708870C86002468861ED
:103F90001A54401C3C28FBD38A617047440100201E
:103FA000F003002070B504211C48FDF747FF1C4CAE
:103FB0004FF4805120701B48FDF740FF60704FF4B4
:103FC00000411948FDF73AFF211FA070087800232F
:103FD000032800D30B700878114A245CD21E0CB958
:103FE000155C1DB1155C022D0DD00FE00F4C54F87F
:103FF00020506D1C44F82050052D07D944F820307E
:104000000124145402E0012C00D11354401CC0B20E
:104010000870032800D30B7070BD0000001401402D
:1040200078000020001001400008014074030020C7
:1040300070B500244FF40065134E04E0641CE4B234
:10404000012001F03FFF29463046FDF7F7FE012829
:1040500003D0C82C10D2002407E0C82CEED30BE00C
:10406000641CE4B2012001F02DFF29463046FDF723
:10407000E5FE18B1F02C04D3012070BDF02CEFD375
:10408000FAE7002070BD00000010014070B586B056
:104090000024104801940294816941F0100181616B
:1040A00080690D4E00F0100004904FF4006002256E
:1040B0000090694603953046FDF7C4FD6802009004
:1040C00001AA012082E8310069463046FDF7BAFDB9
:1040D00006B070BD001002400010014070B5002411
:1040E00000F08AF800F06EF8FFF7A2FF114908709F
:1040F000CC2000F08FF8BE2000F08CF800F052F8D1
:10410000054600F04FF8072800D8012405EB0020F1
:1041100000B23CB102F058FFBDE870406FF00301FF
:1041200003F059B9C04302F04FFFBDE870400249A7
:1041300002F0AABF88000020000080BD10B5FFF784
:10414000A5FF012291020448FDF77DFE00F03AF838
:10415000BDE81040FFF76CBF0010014070B5104D76
:104160004FF48064002221462846FDF76CFE0220B1
:1041700001F0A8FE012221462846FDF764FE0C202E
:1041800001F0A0FE61002846FDF758FE08B10124A9
:1041900000E00024322001F095FE204670BD0000B2
:1041A0000010014070B500255FF00104FFF7D6FF55
:1041B000C001641C40EA5500E4B2C5B2082CF5D930
:1041C000284670BD70B50B4D4FF480640022214627
:1041D0002846FDF738FE40F2EE2001F073FE012282
:1041E00021462846FDF72FFEBDE870400F2001F064
:1041F00069BE00000010014010B5FFF7E3FFFFF7B4
:1042000017FFCC2000F006F8BDE81040442000F075
:1042100001B800002DE9F0410124154F0546A60222
:1042200015F0010F4FEA55054FF0000231463846B0
:104230000BD0FDF708FE022001F044FE01223146BA
:104240003846FDF700FE3C200AE0FDF7FCFD3C206F
:1042500001F038FE012231463846FDF7F4FD022018
:1042600001F030FE641CE4B2082CD9D9BDE8F0811D
:1042700000100140094808B5416941F00101416160
:104280004069002200F00100009011461020FEF766
:10429000DBF8BDE808401020FEF7C8B80010024067
:1042A0002DE9F04F85B000244A480094019402940F
:1042B0000394816941F010018161816901F010016D
:1042C0000491816941F020018161816901F020013F
:1042D0000491816941F004018161816901F0040167
:1042E0000491816941F0080181618069DFF8E8A0EB
:1042F00000F0080041F612060490002231465046B4
:10430000FDF7A1FDDFF8D4904FF4F068002241469C
:104310004846FDF798FDDFF8C8B00022382158461E
:10432000FDF791FD4EF24F000325CDE900056946EA
:104330004846FDF787FCE120CDE900056946504677
:10434000FDF780FC0096022701260397CDE9016462
:1043500069465046FDF776FC41F63000CDE9000491
:10436000694648460294FDF76DFCCDE90054694664
:1043700058460294FDF766FC41F20430CDE9000591
:1043800069465846FDF75EFCCDF800800397CDE9FD
:10439000016469464846FDF755FC4FF40140CDE9FC
:1043A0000004694650460294FDF74CFC0420CDE918
:1043B000000469460B480294FDF744FC3820CDE91F
:1043C0000006CDE9024769465846FDF73BFC05B0BB
:1043D000BDE8F08F001002400008014000100140CD
:1043E000000C0140001401400D4810B50B4901605C
:1043F0000C49416000214FF480428160C0E9031202
:1044000041618161C1610162FDF7A6FE002803D010
:10441000BDE81040FDF74EB910BD0000005400404B
:1044200064010020A08601000F4810B50D4901600D
:104430004FF48271416000218160C1604FF40072CD
:104440000161C0E90512C1610162416281620A2114
:10445000C162FEF709FB002803D0BDE81040FDF75C
:1044600029B910BD00380040B801002010B586B051
:10447000002419480094019402940394049415496B
:10448000059401602321C0E9011440F2E731C0E93D
:1044900003148021C0E90541FEF7DEFB08B1FDF7FA
:1044A00009F94FF48050009069460B48FEF756FC1E
:1044B00008B1FDF7FFF8049404A907480594FEF736
:1044C0008DFB08B1FDF7F6F80348FEF711FC06B0C6
:1044D00010BD0000002C0140100200200C4810B557
:1044E0000A4901604FF4E1314160002181600C22F2
:1044F000C160C0E904128161C161FEF721FF00289B
:1045000003D0BDE81040FDF7D5B810BD003801401C
:10451000580200200C4810B50A4901604FF41651AA
:104520004160002181600C22C160C0E904128161F8
:10453000C161FEF705FF002803D0BDE81040FDF77C
:10454000B9B810BD00440040A00200200C4810B5CE
:104550000A4901604FF4E1314160002181600C2281
:10456000C160C0E904128161C161FEF7E9FE002863
:1045700003D0BDE81040FDF79DB810BD00480040D5
:10458000E8020020FEE7FEE710B5AE2000F050FF85
:10459000002000F04DFF102000F04AFF402000F006
:1045A00047FFB02000F044FF812000F041FFFF20D2
:1045B00000F03EFFA02000F03BFFA62000F038FFF7
:1045C000A82000F035FF3F2000F032FFC02000F0AF
:1045D0002FFFD32000F02CFF002000F029FFD52072
:1045E00000F026FF802000F023FFD82000F020FFFD
:1045F000052000F01DFFD92000F01AFFF12000F087
:1046000017FFDA2000F014FF122000F011FFDB206A
:1046100000F00EFF302000F00BFF8D2000F008FFAF
:10462000142000F005FFAF2000F002FFBDE81040AD
:10463000AFF3008070B5002404F1B000C0B200F008
:10464000F7FE002000F0F4FE102000F0F1FE00253F
:10465000002000F004FF6D1CEDB2802DF8D3641C27
:10466000082CE9DB70BD00002DE9FC5FF74EDFF898
:10467000E0A306F10D0006F1100772780078796862
:104680000091F549DFF8CCB300240125096806F153
:10469000300906F140080B2A7ED2DFE802F0060955
:1046A00049CEFDFCFBFAF9F8F700FFF76DFF3CE09F
:1046B000FFF7C0FF1023E9A200213020009500F091
:1046C0001DFE1023E7A202210020009400F016FE38
:1046D0001023E7A204210020009400F00FFE102315
:1046E000E7A206210020009400F008FED74DED1D42
:1046F000287830B910233C2202217020009400F069
:104700008FFD2878012806D110233C220421702037
:10471000009400F085FD2878022806D110233C2261
:1047200006217020009400F07BFD7078401C74E03E
:10473000C64DED1D2878F8B96878002871D010238F
:104740003C2202217020009400F06AFD6878012864
:1047500006D11023202204217020009400F060FD77
:104760006878022806D110232022062170200094A8
:1047700000F056FD287868702878012820D16878E4
:10478000012854D010233C2204217020009400F012
:1047900047FD687840B900E040E010232022022164
:1047A0007020009400F03CFD6878022806D11023A8
:1047B000202206217020009400F032FD28786870D5
:1047C000287802281ED16878022821D010233C22A4
:1047D00006217020009400F023FD687830B9102382
:1047E000202202217020009400F01AFD6878012830
:1047F00006D11023202204217020009400F010FD27
:1048000028786870287858B1012810D0022805D17E
:10481000B078012802D1B47008207070BDE8FC9F08
:10482000FFE7B0780128F9D1B4700320F5E7B0783C
:104830000128F3D1B4700420EFE7F078DFF850924C
:1048400000287DD039600191009802F01BFDDFF84F
:104850004482404505DADDE9001002F013FD4045D1
:1048600023DB10238CA202212820009400F046FDB7
:104870008A49386802F008FC02F0F0F902460B465B
:1048800087A18948FBF7E2FC102306E0F0E3F0E3A0
:104890005DE35BE206E2A8E11FE1834A022100201A
:1048A000009400F02BFD38687860684FD9F800104C
:1048B00018373960786802F033FB1AD0102376A2DB
:1048C00006212820009400F019FD786802F0C6F94E
:1048D000024675480B4672A11030FBF7B7FC724ACE
:1048E0001023103206210020009400F007FD3868E4
:1048F00078609AF8000002F07FFB544F01462037A1
:104900003860786802F00CFB0DD038684FF0100367
:10491000B0F17E5F00947DD064A20221482000F0B7
:10492000EDFC386878609BF8000002F065FB474FAB
:10493000014628373860786802F0F2FA0FD000E0BC
:1049400015E038684FF01003B0F17E5F009476D028
:1049500056A20621482000F0D1FC38687860B07873
:1049600001287FF45BAFB4707570F47056E7F57092
:10497000FFF760FE002110234EA20846009400F0CD
:10498000BDFC35484549006802F07EFB02F066F93F
:1049900002460B4642A14448FBF758FC1023424A0A
:1049A00002210020009400F0A9FC102342A2002163
:1049B0004820009400F0A2FC102340A20421002013
:1049C000009400F09BFCD9F8000002F047F9024681
:1049D00035480B4632A11030FBF738FC324A102321
:1049E000103206210020009400F088FC102335A22C
:1049F00004214820009400F081FC102332A20221FF
:104A00003020009400F07AFC9AF800004FF0100378
:104A1000012800E018E0009412D024A202214820CE
:104A200000F06CFC9BF800004FF01003012800948C
:104A300008D01EA20621482000F060FC8FE749E064
:104A400022A2EBE721A2F5E720A266E7C40000203E
:104A50005400002055000020640000204D656E7554
:104A600000000000506172616D6574657220000085
:104A70004D6F746F7220436F6E74726F6C00000024
:104A80004D61676E65742053616D706C6500000048
:104A9000680000206F12833A200000000000C84226
:104AA000252E326600000000D00300204552524FF0
:104AB00052000000506F73004F43310054656D7019
:104AC000000000004F4332002500000020204F4B23
:104AD00020000000AFF20C023BE7317931B1F74F13
:104AE0007978884265D0002850D056E03571FFF7BC
:104AF000A1FD1023AFF2880200210846009400F0C7
:104B0000FDFB1023EEA202210020009400F0F6FB32
:104B1000EE4F387830B91023EDA2022150200095D5
:104B200000F0ECFB3878012806D11023EAA202211C
:104B30005020009500F0E2FB1023E9A204210020A0
:104B4000009400F0DBFBE948E9A10268E948FBF7C3
:104B50007DFB1023E74A04215020009400F0CEFB97
:104B60001023E5A204216420009400F0C7FB102369
:104B7000E2A206210020009400F0C0FB1023E1A275
:104B800006215020009400F0B9FB12E01023D0A2BF
:104B900002215020009500F0B1FB3878012806D1A1
:104BA0001023CDA202215020009500F0A7FB3878F9
:104BB0007870B07801287FF4D9AEC04DB4703471EC
:104BC000287830B91023C2A202215020009400F0AE
:104BD00095FB2878012806D11023BFA2022150207E
:104BE000009400F08BFB052017E6DFF8D0A24FF011
:104BF000060870BB3079E8B14F46D7E9000188421A
:104C000012D01023C0A204215020009400F076FBA3
:104C1000B7A1B8483A68FBF719FB1023B54A04213D
:104C20005020009500F06AFB38687860B078012861
:104C300010D01AE0AD483571ADA10268AD48FBF760
:104C400005FB1023AB4A04215020009500F056FBD1
:104C5000ECE70AE0B47034711023A64A0421502016
:104C6000009400F04BFB86F801809AF800000128C0
:104C7000A1D1C9F800504F461023A3A2042150200F
:104C8000009400F03BFB9AA19A483A68FBF7DEFAE1
:104C90001023984A04215020009400F02FFB86F83E
:104CA0000180BBE5854F30793F1F28B1387879788E
:104CB000884229D048B116E035713C707C701023D1
:104CC00006218EA2002000951CE010238BA2062155
:104CD0000020009500F012FB10238AA2062150202C
:104CE000009400F00BFB387801280DD1102383A22B
:104CF00006210020009400F001FB102381A2062170
:104D00005020009500F0FAFAB0780128C9D138781F
:104D100078B10128C5D17D48B470347105706748F9
:104D20006A49007808707148D9F8001001600720BE
:104D300073E57648B4703471047060480470447050
:104D4000C9F80050C9F80450757067E57079E0B390
:104D500039608946009802F095FADFF8B481404541
:104D600005DA4846009902F08DFA40451DDB102314
:104D7000AFF2DC2202215020009400F0BFFA654916
:104D8000386802F081F901F069FF02460B46AFF284
:104D9000F0215848FBF75AFA1023564A02212820DE
:104DA000009400F0ABFA386878609AF8000002F0DE
:104DB00023F9424F014613373860786802F0B0F8A3
:104DC00010D03868B0F17E5F00E02FE04FF01003A4
:104DD000009470D0AFF22C320621082000F08EFA39
:104DE000386878609BF8000002F006F9334F0146FE
:104DF0001B373860786802F093F80ED038684FF0AF
:104E00001003B0F17E5F009456D0AFF260320621FD
:104E1000482000F073FA38687860B078012894D19F
:104E20003A480470B47075707471F7E47571FFF7E7
:104E300001FC0021102338A20846009400F05EFA1D
:104E4000102338A202210020009400F057FA10230A
:104E5000AFF28C3202215A20009400F04FFA102356
:104E600032A204210020009400F048FA102331A25D
:104E700004214020009400F041FA9AF800004FF01D
:104E800010030128009413D0AFF2E032062108206D
:104E900000F034FA9BF800004FF010030128009452
:104EA0004CD0AFF2F8320621482000F027FAB4E7E0
:104EB000AFF2E832EAE744E046E00000D10000202B
:104EC00052756E204D6F64653A0000000D010020A0
:104ED00053544550000000004C4F4F50000000005C
:104EE00052756E20537465703A0000002001002056
:104EF00025640000D00300206D6D000043616E63E7
:104F0000656C00004F4B0000202000000C010020C9
:104F10006F12833A0000C84252756E6E696E672E3A
:104F20002E2E0000506F733A000000004F43313ABC
:104F3000000000004F43323A00000000AFF274421C
:104F4000B1E7AFF2784247E7AFF280425FE7B0796E
:104F5000C8B39E4FD7E90001884216D01023AFF2A4
:104F6000C84202215820009400F0C8F9AFF2800135
:104F700097483A68FBF76AF91023954A02215020B6
:104F8000009500F0BBF938687860B07801287FF4AC
:104F9000EDACB470B4711023AFF294020221502032
:104FA000009400F0ABF98948AFF2BC010268884870
:104FB000FBF74CF91023864A02215020009400F0A0
:104FC0009DF9092029E4FFE7B571FFF733FB0021C4
:104FD000102380A20846009400F090F9102380A2CC
:104FE00002210020009400F089F910237FA2022101
:104FF0006420009400F082F910237DA20421002097
:10500000009400F07BF97C487049C2780A604A60DD
:105010004079C8F80000AFF22811C8F804006C48C5
:10502000FBF714F910236A4A02215020009500F082
:1050300065F9AFF244116648D8F80020FBF706F98D
:105040001023634A04215020009400F057F91023E4
:10505000AFF2581206210020009400F04FF91023FF
:10506000AFF2601206215020009400F047F98CE75F
:1050700050E0FFE75549B07908310A68D8B3D8F84D
:105080000400824219D01023AFF2F45204215820B8
:10509000009400F033F9AFF2A8114D48D8F8002081
:1050A000FBF7D4F810234A4A04215020009500F061
:1050B00025F9D8F80000C8F80400B07801287FF47A
:1050C00055ACB470B4711023AFF2C4120421502057
:1050D000009400F013F9AFF2E8113D48D8F8002031
:1050E000FBF7B4F810233A4A04215020009400F052
:1050F00005F90A2078E5FFE7B571AFF20C213448D5
:10510000FBF7A4F81023324A04215020009500F048
:10511000F5F8D2E73746B0792C4E2D3E28B13078DD
:105120007178884232D060B11BE0BD713470747008
:105130001023AFF2382206210020009500F0DEF89F
:1051400024E01023AFF24C2206210020009500F04D
:10515000D5F81023AFF2542206215020009400F01D
:10516000CDF8307801280FD11023AFF2702206213C
:105170000020009400F0C2F81023AFF2782206213C
:105180005020009500F0BAF830787070B978384641
:10519000012994D1317861B1012990D10B498470F2
:1051A00084710A781449CA7098F800204A717D7099
:1051B00077E511498470054A8471CB781360536098
:1051C0004979C8F80010C8F80410F0E7FC00002086
:1051D000D003002053616D706C652053657400002E
:1051E000496E74657276616C3A0000006D73000060
:1051F0004465657074683A006C00002010B5044680
:10520000B031C8B200F014F9102040EA141000F0D8
:105210000FF904F00F00BDE8104000F009B90000DC
:105220002DE9F0418046203A002406980E46D7B278
:10523000B8F17F0F02D9B61CA046F6B2102B11D0E0
:1052400031464046FFF7DAFF2A4907EB470001EBFA
:105250004005285D00F003F9641CE4B2062CF8D385
:10526000BDE8F081244D20B30128F9D131464046F4
:10527000FFF7C4FF04EB0710285CC043C0B200F086
:10528000EEF8641CE4B2082CF4D3761CF1B240466C
:10529000FFF7B4FF5FF0000404EB07102844007A26
:1052A000C043C0B200F0DBF8641CE4B2082CF3D3B6
:1052B000D6E731464046FFF7A1FF00BF04EB0710D9
:1052C000285C00F0CCF8641CE4B2082CF6D3761C01
:1052D000F1B24046FFF792FF5FF0000404EB0710C5
:1052E0002844007A00F0BBF8641CE4B2082CF5D323
:1052F000B6E700007C740008A47600082DE9F843A6
:10530000994617460E4604460025DDF820800FE03A
:105310004B4631462046CDF80080FFF781FF083428
:10532000E4B2782C02D90024B61CF6B26D1CEDB2A2
:105330007A5D002AECD1BDE8F883704770B5114E54
:10534000002210213046FCF77EFD0A2000F0B4FD5B
:10535000102000F003FC00F017F8044600F014F8E9
:10536000054600F011F8014645EA042041EA002410
:105370000A2000F0A1FD012210213046FCF763FD58
:10538000204670BD0008014070B5134E0022202158
:105390003046FCF758FD0024012220213046FCF75E
:1053A00052FD012000F088FD6806050E40213046C0
:1053B000FCF744FD08B145F00105002220213046EC
:1053C000FCF741FD012000F077FD641CE4B2082CDD
:1053D000E2D3284670BD00000008014070B50C4DB6
:1053E000002210212846FCF72EFD232000F0B6FBFA
:1053F0005FF00004FFF7C8FF641CE4B2042CF9D38B
:105400002846BDE8704001221021FCF71CBD0000B9
:10541000000801400148FDF7B7BA0000B8010020BC
:1054200010B5406A0021C187C186FDF7ABFA10BDF7
:1054300010B5044600F0DCFD782000F0ABFD00F074
:105440005BFD002000F0A6FD00F056FD204600F0B8
:10545000A1FD00F051FDBDE8104000F0E9BD10B520
:10546000044600F0C5FD782000F094FD00F044FDF6
:10547000402000F08FFD00F03FFD204600F08AFD47
:1054800000F03AFDBDE8104000F0D2BD70474FF08B
:10549000E0210428086903D020F004000861704767
:1054A00040F00400FAE7FCF769BF30B58FB028215F
:1054B0006846FAF7A2FF14210AA8FAF79EFF012115
:1054C0000804CDE900100024029402250491CDE9DE
:1054D00007504FF4E01009906846FDF7C3F860B933
:1054E0000F20CDE90A058020CDE90C0402210AA88D
:1054F0000E94FCF7DBFF002801D0FCF7DBF80FB0BF
:1055000030BD70470148FDF798BC00001002002034
:10551000F0B502681C4B1D4D1D4E1E4F1E4C4FF02A
:10552000804C984209D0A04207D0604505D0A842DF
:1055300003D0B04201D0B84204D122F0700E4A68C4
:1055400042EA0E02984209D0A04207D0604505D039
:10555000A84203D0B04201D0B84203D122F4407532
:10556000CA682A434D6922F080022A4302608A6891
:10557000C2620A688262984201D0A04201D10969E0
:10558000016301214161F0BD002C01400004004095
:1055900000080040000C00400034014010B5846851
:1055A00042EA032224F47F440A432243826010BD6E
:1055B000826822F070020A4342F00701816070475E
:1055C00010B5036A046A24F001040462846924F0BB
:1055D000F00444EA021423F00A020A4384610262DE
:1055E00010BD10B5036A046A24F0100404628469D3
:1055F00023F0A00324F4704444EA023243EA011188
:105600008261016210BD000070B586B010480024B0
:105610000294816941F00801816180690D4E00F0BA
:10562000080004904FF420400090012002250190D2
:10563000694603953046FCF705FB6803CDE9000495
:10564000694603953046FCF7FDFA06B070BD0000D0
:1056500000100240000C01402DE9F05F054617469E
:1056600000200E46444A044601461154401CC0B274
:105670000528FAD3002280214048FCF7E4FB64208F
:1056800000F000FC17B145F0800501E005F07F0552
:10569000DFF8EC904FF4005A012251464846FCF7DF
:1056A000D2FB00274FF4804B0022D046514648469B
:1056B000FCF7C9FB280601D5012200E000224FF4C7
:1056C00000414846FCF7BFFB6806050E0122C246B2
:1056D00041464846FCF7B7FB142000F0D3FBDFF847
:1056E0009880484698F80010490088F800105946FC
:1056F000FCF7A4FB28B198F8001041F0010188F8EC
:1057000000107F1CFFB2082FCED30027C84600220E
:10571000D14651464046FCF796FB002E01DA0122A5
:1057200000E000224FF400414046FCF78CFB76007D
:10573000012249464046FCF786FB142000F0A2FBFC
:10574000640059464046FCF779FB08B144F0010477
:105750007F1CFFB2202FDAD30748210E01220570EB
:105760004170210C8170210AC1700471BDE8F05FA5
:1057700080210248FCF767BBBC00002000100140FC
:10578000000C014010B5406A0021C185C184FDF7BD
:10579000A0FC10BD70B5446A2068406994F84110BF
:1057A000C0F3C0100025212904D118B1E58420469A
:1057B00000F08EF82068406994F84210C0F3801021
:1057C000222904D118B1E585204600F05AF8606C12
:1057D00040F0100060642046FDF77BFC70BD10B502
:1057E0000146406A096809684FF0000289062ED414
:1057F000C28501680C3151E8003F23F4807341E811
:105800000034002CF5D10168143151E8003F23F039
:10581000010341E80034002CF5D10168143151E84E
:10582000003F23F0400341E80034002CF5D1202153
:1058300080F84210016B012909D101680C3151E84F
:10584000003F23F0100341E80034002CF5D14263FF
:10585000016B012902D0FDF769FE10BD818DFDF7B6
:1058600037FC10BD10B5406A01214163016B01296D
:1058700002D0FDF75CFE10BD818D4908FDF728FCC4
:1058800010BD01680C3151E8002F22F4907241E8FC
:105890000023002BF5D10168143151E8002F22F0CC
:1058A000010241E80023002BF5D1016B012909D148
:1058B00001680C3151E8002F22F0100241E800236A
:1058C000002BF5D1202180F84210002101637047A0
:1058D00001680C3151E8002F22F0C00241E800239A
:1058E000002BF5D1202180F84110704708B590F8C1
:1058F0004210222901D0022008BD82684FF4805353
:105900009A4201D1016921B1816A9A421BD04AB100
:105910000AE00268816A5268C2F308020A80816A5A
:10592000891C08E0026972B10268526802F07F02C5
:105930000A70816A491C8162C18D491E0904090CE3
:10594000C18503D01BE002685268F1E70168CA68AC
:1059500022F02002CA600168CA6822F48072CA601C
:1059600001684A6922F001024A61202180F8421050
:1059700000214163026B012A03D0FDF7D7FD00200F
:1059800008BD016301680C3151E8002F22F01002BC
:1059900041E80023002BF5D101680A68D20602D540
:1059A0000A6849680091818DFDF792FBE7E70000E6
:1059B00070B5044600680169E26821F44051114362
:1059C00001612169A0680843616908432168CA68C8
:1059D00041F20C639A430243CA6020684169A2699C
:1059E00021F44071114341611E492068884202D16F
:1059F000FCF702FE01E0FCF7EFFD00EBC00101EB5C
:105A00000012606864218000B2FBF0F3B3FBF1F395
:105A10006FF018067343B2FBF0F5B2FBF0F605EB3E
:105A20008305322303EB0515B5FBF1F5B6FBF1F663
:105A300005F0F00505EB0615B2FBF0F6B2FBF0F051
:105A4000B0FBF1F06FF01802504306EB800003EB5F
:105A50000010B0FBF1F0216800F00F0028448860CE
:105A600070BD00000038014038B58162044682856F
:105A7000002013466064222284F84220E56B1B4A12
:105A8000AA62E56B1A4AEA62E56B1A4A2A63E26B7C
:105A900050630A462168E06B091DFCF79BF82068FB
:105AA000016840680090206948B120680C3050E8D7
:105AB000001F41F4807140E80012002AF5D12068EF
:105AC000143050E8001F41F0010140E80012002AA4
:105AD000F5D12068143050E8001F41F0400140E843
:105AE0000012002AF5D1002038BD0000DF57000861
:105AF000655800089557000810B50948FDF7EAFAFF
:105B000008480068800609D50648001D0068064957
:105B1000C0B20870BDE8104000F0DCBB10BD000052
:105B200058020020003801400000002010B5054850
:105B3000FDF7D0FABDE81040062203490148FDF701
:105B4000A0BA0000A00200203C0000200148FDF7A0
:105B5000C1BA0000E8020020FEE7000070B5134E55
:105B600005460024280601D5012200E000228021FC
:105B70003046FCF768F96806050E0A2000F0A2F925
:105B8000012220213046FCF75EF90A2000F09AF944
:105B9000002220213046FCF756F90A2000F092F945
:105BA000641CE4B2082CDDD370BD00000008014085
:105BB0002DE9F041124F15460E46044600221021F1
:105BC0003846FCF740F90C20711E00EA840001F011
:105BD0000301084340F04000FFF7C0FF002405E048
:105BE0002878FFF7BBFF641CE4B26D1CB442F7D306
:105BF0003846BDE8F04101221021FCF724B900002D
:105C0000000801402DE9F047DFF87CA000251F4C7B
:105C100088468146CAF804506F1CFEB211E000BFEE
:105C200054F8261054F8250001F0FAFA07D254F877
:105C3000250054F8261044F8251044F82600761C58
:105C4000F6B2142EECD3FDB2132DE5D3A9F1010069
:105C5000C5B25646DAF8040006E000BF54F8251035
:105C600001F028F86D1CEDB24545F7D30446A8EBCA
:105C70000900401C01F0A8F90146204601F08EF809
:105C80007060BDE8F08700007C00002080030020E9
:105C90000C4810B50168012913D10B4C002101609B
:105CA0002078142801D2012100E000214143217015
:105CB0000420FBF711FD054A217842F82100491C18
:105CC000217010BD100000207C0000208003002007
:105CD000490050EAC12018BF04204A0D18BF40F007
:105CE000010040F2FF72B2EB515F08BF40F00200CA
:105CF000012808BF052070470907090E002804DBAA
:105D000000F1E02080F80014704700F00F0000F16F
:105D1000E02080F8141D704730380A2801D2012095
:105D200070470020704700002DE9F04700F098F917
:105D300049480027494C0168494E01290CD10760A8
:105D4000012202213046FCF77EF8072204F11801F7
:105D50004448FDF7EDFBA07043480168D9B10760E6
:105D6000FEF782FCFEF7BAF9606110210520FFF70B
:105D700049FF6060A16805468946E06801F082FA43
:105D800080464946284601F07DFA414601F006F872
:105D9000206100F08DFAFFF77BFFFBF7D5FB33485E
:105DA000334D4178297181786971C178A971007981
:105DB000E8712F72606801F0E7F8687220212D48C1
:105DC000FCF73CF8207001212B48FCF737F8607095
:105DD0002A4C2B4D4FF4805720784FF4006818B1AF
:105DE00003280BD1287830BB012239463046FCF716
:105DF0002AF8012241463046FCF725F82078012890
:105E000009D1002239463046FCF71DF801224146EF
:105E10003046FCF718F82078022809D101223946CB
:105E20003046FCF710F8002241463046FCF70BF8EC
:105E3000207803280ED1287801280BD1002239467A
:105E40003046FCF700F841463046BDE8F0470022F6
:105E5000FBF7F9BFBDE8F0873000002054000020B8
:105E600000080140A0020020200000203C0000208B
:105E70002C04002000100140000C01408C00002088
:105E80008D00002000E000BF401EFCD270470000E3
:105E900010B56FF00400FFF7FAFA044804490068EF
:105EA000B0FBF1F00349087010BD00005000002065
:105EB00000127A0073000020002100E0491C81429A
:105EC000FCDB70470B49097848434FF0E0214861FB
:105ED00000228A61086940F0010008610869C3076F
:105EE00001D0C003FAD5086920F0010008618A6179
:105EF000704700007300002010B50E4C0022802176
:105F00002046FBF7A0FF00F03FF801224021204689
:105F1000FBF799FF00F038F8002240212046FBF7FC
:105F200092FF00F031F820460122BDE810408021A8
:105F3000FBF789BF000C014000B585B0002002903E
:105F40000F48816941F008018161816901F0080110
:105F50000491816941F0080181618069694600F01E
:105F600008000490C02000901120019003200390AD
:105F70000448FBF767FE00F05BF805B000BD0000C9
:105F800000100240000C01400020401CC0B20A2852
:105F9000FBD3704770B5154E05460024280601D581
:105FA000012200E0002280213046FBF74CFFFFF782
:105FB000EBFF012240213046FBF745FFFFF7E4FFEE
:105FC000002240213046FBF73EFF072C04D101227E
:105FD00080213046FBF737FF6806050EFFF7D4FF38
:105FE000641CE4B2082CD9D370BD0000000C014041
:105FF00010B50E4C012280212046FBF724FF012220
:1060000040212046FBF71FFFFFF7BEFF0022802143
:106010002046FBF718FFFFF7B7FF0022402120467C
:10602000FBF711FFBDE81040FFF7AEBF000C0140C9
:1060300010B50A4C002280212046FBF704FF012204
:1060400040212046FBF7FFFEFFF79EFF204601227E
:10605000BDE810408021FBF7F6BE0000000C0140B7
:106060002DE9F04F674C02274FF0010E20780128F0
:1060700003D1654981F800E02770644894F801C0B5
:10608000634E0378634D6448DFF890916449654A34
:10609000DFF894A19B1E4FF00A0BBCF1010F62D1F7
:1060A000092B5FD2DFE803F0055E12202D5E3A4730
:1060B000540096F800C0BCF1020F02D20CF1010CA2
:1060C00001E04FF0000C86F800C04BE095F800C0EE
:1060D000BCF1000F05D04FF0000C00BF85F800C0E8
:1060E00040E04FF0010CF9E7D0F800C0BCF1010F1F
:1060F00002D9ACF1010C01E04FF00F0CC0F800C068
:1061000030E099F80080B8F1000F04D04FF000089B
:1061100089F8008026E04FF00108F9E7D1F800C0C7
:10612000BCF1050F04D9ACF1010CC1F800C019E0B5
:10613000C1F800B016E0D2F800C0BCF10A0F02D9D5
:10614000ACF1010C01E04FF0140CC2F800C009E002
:106150009AF80080B8F1000F13D04FF0000800BF8C
:106160008AF80080677094F802C0BCF1010F44D136
:10617000092B41D2DFE803F008400F161F402931F8
:106180003A004FF00108EBE7307810B1401E307054
:1061900032E0377030E0287810B1002028702BE012
:1061A0000120FBE701680F2902D2491C016023E0AE
:1061B000C0F800E020E099F8001021B15FF0000184
:1061C00089F8001018E00121FAE708680A2801D2CE
:1061D000401C00E0052008600EE01068142802D280
:1061E000401C106008E0C2F800B005E09AF800100A
:1061F00029B100218AF80010A770BDE8F08F0121B5
:10620000F8E7000075000020C6000020C50000204F
:10621000CB000020D1000020F4000020CD000020A1
:10622000FC00002004010020CF000020FCF7AEF8A5
:10623000FFF73BF9FEF734F8FEF71CF8FEF716F906
:10624000FEF7D2F8FEF7F0F8FEF748F9FEF762F92C
:10625000FEF77CF9FFF71CFEFFF76EFEFEF794F9E0
:106260000D4C012211032046FBF7EDFD0122D10266
:106270002046FBF7E8FDFDF709FFFDF75FFFFBF7A1
:10628000BFF8FFF7C1F900F047F8FDF775FE00BF52
:10629000FFF74AFDFCE70000000801400348002129
:1062A00041708170C170FDF767BE0000440100209D
:1062B00007484178012902D18178491C8170C17851
:1062C000002904D08078884201D3FFF7E7BF7047E8
:1062D000440100200346094800B500783C2807D255
:1062E0000A2000F00DF818465DF804EBFBF788B9BA
:1062F000FFF7D4FF5DF804EBFDF73EBE440100203C
:10630000002805D0034901224A7000228A70C87013
:10631000704700004401002010B501220421002034
:10632000FFF79AF9012231491020FFF795F9012270
:106330000A211120FFF790F9012210211420FFF704
:106340008BF9012210211520FFF786F9284C012234
:1063500020206168FFF780F9012200212120FFF74A
:106360007BF9012200212320FFF776F90122242066
:106370006169FFF771F901222620A169FFF76CF925
:1063800001222520E168FFF767F901222720216912
:10639000FFF762F901222A20E169FFF75DF9012286
:1063A0002820216AFFF758F9012210212B20FFF73E
:1063B00053F9012243F6FF712C20FFF74DF901221A
:1063C0002D20A168FFF748F901220A496C20FFF748
:1063D00043F9012200216D20FFF73EF90122BDE8BB
:1063E000104005497020FFF737B90000020E070082
:1063F0008C000020C30001001E000CC410B5002951
:106400000AD00878002807D005487844FAF7D4FB6A
:10641000002801D0002010BD0248784410BD0000C3
:106420003E1900003619000021F00042A2F160522E
:10643000B2F5801F01F0004328BFD2F17F6C0BD969
:106440005FEA001C43EAC20242EB507018BF70477B
:1064500028BF20F001007047B2F5801FBCBF18466E
:1064600070474FEA410C1CF5001F02D2084600F0AD
:10647000D2BE70B500F0B4FA00000089FFF7F6BF95
:106480004FF00040A0F580007047000010B591EA81
:10649000030F48BF83F0004300F1FE82841A71EBC2
:1064A000030C05D2121943EB0C03001B61EB0C012A
:1064B000DFF824E14FEA1154A4EB135C1EEA430F0A
:1064C00018BF9EEA445F73D023EA0E03DCF1200E6E
:1064D00021EA045143F4801332D322FA0CFE10EB6C
:1064E0000E0023FA0CFE41EB0E01CCF1200E03FA54
:1064F0000EFE10EB0E0051F10001B1F5801FCCF142
:10650000200E32D201EB045112FA0EF2BDE8104017
:1065100058BF7047401C38BF5FEA420218BF70473F
:10652000002814BF20F0010041F100014FEA4103AF
:1065300013F5001F38BF7047A1F1C04100F09EBAAB
:10654000012A43EB0302ACF1200CDCF11F0E32BF39
:106550004FF0000E23FA0CF310EB030041EB045153
:10656000B4EB115FD0D0A1EB045101F580114908C3
:106570005FEA300001EB04510ED350F1000038BF48
:1065800012FA0EFE08D1BDE81040C9E7401C38BF22
:106590005FEA4202CAD1C3E7BDE810404FEA4103B7
:1065A00013F5001F38BF7047A1F1C04100F066BA73
:1065B0009EEA445F08D011EA5E0FBDE8104004BFB8
:1065C00001F0004100207047BDE8104070B500F0B8
:1065D00007FA00BF64FBBE3E0000E0FF2DE9C041AA
:1065E00030B4DFF8A0C23CEA111418BF3CEA13141F
:1065F00000F0EC8081EA03051CEA111444EAD5742A
:1066000018BF1CEA131500F0C780A4EB05044FF077
:10661000004545EAC12145EAC32341EA505143EA16
:10662000525304F17F74994204F500344FEAC020BC
:106630004FEAC22208BF904200F09C804FEA1365E7
:106640000FF24016765D4FEA134506FB05F7C7F1DA
:10665000807706FB07F74FEAD737A7FB0368764238
:10666000C8F58038A7FB06CE38BFA8F1010807FBA4
:1066700008E64FF0000EA6FB028CE6FB03CEDCF131
:10668000000CCEF1004E38BFAEF1010EA6FB0C5847
:106690004FF000074FF00005E6FB0E87A1FB08C690
:1066A000A0FB07CE16EB0E0645F10005E1FB0765E2
:1066B00015F1E04E7EBFA4F580345FEA46066D41D9
:1066C00016F1800745F100054FEA17274FEA0666E5
:1066D00047EA0567A6F1DE46B6F1805F4FEA152569
:1066E0001FD9384624F0010C05EBC471BCF1FE6FD4
:1066F00001EB0C1102D8F0BCBDE8008124425CBF64
:1067000001F5801E9EEAC47F02D4F0BCBDE8008182
:10671000244238D4F0BCA1F1C041BDE8004100F0F2
:10672000ADB94FEAD22242EA43524FEAD323A7FB44
:1067300002864FEAD02040EA415007FB03661EEA7A
:106740000E0F4FEAD12105FB026658BFA6EB00569B
:10675000B6EB00564FEA520E4EEAC37E18EB0E0E11
:1067600056EB530EBDD518EB02085E417F1C55F168
:106770000005B6E74FF480154FF000074FF0000614
:106780004FF00008ADE7F0BC4FF0000001F1C04150
:1067900001F00041BDE8008111EA0C1F0CEA13155D
:1067A00000D00CE013EA0C1F00F025804FF0000031
:1067B000F0BC81EA030101F00041BDE80081F0BCBA
:1067C000BDE8004181EA030100F058B9F0BCBDE822
:1067D000004170B500F004F9097EFC3E00F007B8F6
:1067E00081EA03014FF0000001F00041704781EAA7
:1067F000030100F043B9F0BCBDE800414FF00000D8
:1068000021497047FFFDFBF9F7F5F4F2F0EEEDEBEF
:10681000E9E8E6E4E3E1E0DEDDDBDAD8D7D5D4D39E
:10682000D1D0CFCDCCCBCAC8C7C6C5C4C2C1C0BFEA
:10683000BEBDBCBBBAB9B8B7B6B5B4B3B2B1B0AFF0
:10684000AEADACABAAA9A8A8A7A6A5A4A3A3A2A1D4
:10685000A09F9F9E9D9C9C9B9A999998979796958F
:1068600095949393929191908F8F8E8E8D8C8C8B2B
:106870008B8A8989888887878685858484838382B3
:10688000828181800000FF070000F87FDFF848C1A7
:1068900070B51CEA111E1EBF1CEA13159EEA0C0FF0
:1068A00095EA0C0F00F06F8081EA030423EA4C1391
:1068B0004EEAD47E21EA4C1141F4801143F4801356
:1068C000AE44A1FB024CA0FB0365AEF17F7E3619FE
:1068D00055EB0C05A1FB034C4CF10003A0FB021C83
:1068E00016EB0C06654153F10003094218BF46F050
:1068F000010613F4007F0BD14FEA03314FEA053054
:10690000340341EA155140EA16506FF003020AE0E1
:106910004FEAC3214FEAC520F40241EA555140EA4B
:1069200056506FF0020202EB2E4201EB025585EA4F
:10693000CE710AD05FEA440C18BF24F0004450F135
:10694000000041F1000120EAD47040F2FE7C624573
:1069500000D270BDA84214BF4FF080444FF04044B5
:10696000002E08BF0024BEF1806FA8BFA1F1C04176
:10697000BDE8704080F282804FF0000001F1C0411C
:1069800001F0004170479EEA0C0F0CEA131518BF86
:1069900095EA0C0F06D04FF0000081EA030E0EF0CE
:1069A000004170BD00F01CF88900013E00F007B8FE
:1069B00000F009B84FEA430C5FEA5C5C08D081EA5A
:1069C000030100F05BB84FEA410C5FEA5C5CF6D172
:1069D0004FF00000014970470000FF070000F87FFA
:1069E0000EF1020E2EF0030E5EF8046B364205D453
:1069F000012A43EB030515F5001F12D8012841EBCE
:106A0000010C1CF5001F0CD80ED14FEAD17C15F5F6
:106A1000001F0CEB4C0C0CF1020C08BF4CEBD37CB0
:106A200004E04FF0080C01E04FEAD37C0CEB4C057E
:106A300026FA05F606F00706B6F1040C06D20EEBB0
:106A4000860CBDE870404CF0010C6047DFE80CF0AC
:106A5000090B02024FF000414FF00000A1F50021A8
:106A600070BD19461046012851EB010418BFD4F53A
:106A7000001484BF002001F0004170BD0808A0F59B
:106A800000114FEA3101704710B591EA030F48BF7A
:106A900083F000433FF502AD841A71EB030C07D27B
:106AA00012198CF0004C43EB0C03001B61EB0C0142
:106AB000DFF8A4E14FEA1154A4EB135C1EEA430F84
:106AC00018BF9EEA445F00F0B08023EA6E03524292
:106AD00021EA0451C3EB6E0338BF5B1EDCF1200ECC
:106AE00025D322FA0CFE10EB0E0043FA0CFE41EB0C
:106AF0000E01CCF1200E03FA0EFE10EB0E0051F148
:106B00000001CCF1200E29D412FA0EF201EB04514F
:106B1000BDE8104058BF7047401C1CBFB2F1004F89
:106B2000704700280CBF491C20F00100704712EB91
:106B3000020E43EB030218BF4FF0010E4EEA420271
:106B4000ACF1200CDCF11E0E54D943FA0CFE10EB14
:106B50000E0051F1FF31CCF11E0ED5D50EF1010E14
:106B600012FA0EFE404141EB010101EB445C5FEA89
:106B70005C5C10D910EBDE7001EB045138BFBEF144
:106B8000004FBDE8104018BF704700280CBF491CDB
:106B900020F00100704730D24FEAD42C11F50011DB
:106BA00024F400641BD0B1FA81F20B3AA41AA41E9B
:106BB000D2F12003914030FA03F31943904001EBE6
:106BC000CC71002C01EB0451BDE81040A8BF704708
:106BD00001F1C0414FF0000001F000417047B0FAF0
:106BE00080F310FA03F100D110BDE41A173C4805F8
:106BF000C90AE4E701EB045110BD491001EB04514F
:106C0000BDE810404FEA300002E04FF0000170474D
:106C10004A0008BF0042F8D0B2F5001F28BF7047F5
:106C200001F000414FF0000070479EEA445F07D03A
:106C300011EA5E0FBDE8104004BF0021002070473C
:106C4000BDE8104070B5FFF7CBFE00BF40DFF63E59
:106C500083F00041104670470000E0FF43004FEA18
:106C6000D30C4FEA3C0C43401FBF40070CF160516E
:106C700013F0FE4F70471CF0006F03D100200CF0A2
:106C8000004170470CF0004343EA507010B540EAF1
:106C9000CC0000F07AFA00BF000000924FEA000139
:106CA000FFF7ECBE4FF000414FF00000A1F50021CE
:106CB0007047000090EA010F48BF81F0004100F1E9
:106CC000E882421A3CBF801A89184FEAD0524FF02E
:106CD0007F4C1CEA410FA2EBD15318BF9CEA026F14
:106CE00000F03B804FF0004C4CEA00204CEA0121C0
:106CF00021FA03FC10EB0C0C1ED202F1FF325FEA0A
:106D00001C2040EBC25038BF70471CF07F0F4FEA89
:106D1000400C18BFBCF17F4F38BF7047C3F1200350
:106D2000994008BF20F00100BCF17F4F38BF704789
:106D3000A0F1C04000F06FBA4FEA3C00000A40EBFF
:106D4000C25028BF1CF0FF0F4FEA400CE6D018BF1E
:106D5000BCF17F4F38BF7047EAE79CEA026F05D06D
:106D600010EA5C0F08BF00F00040704710B500F05B
:106D70000CFA00BF64FBBE3E014800F0FABA00BF47
:106D80000000C07F401058BFC0F14040491058BFBC
:106D9000C1F140418142EFF3008070474FF47F0C16
:106DA0001CEAD0121EBF1CEAD11392EA0C0F93EA20
:106DB0000C0F00F0858090EA010F48BF42F480720A
:106DC00040F4000C41F400002CF07F4120F07F40A3
:106DD00000B58142A2EB03020FF2081CACEB504E4F
:106DE000C0F100009EF800E04FEA4E0E00FB0EFCE2
:106DF00038BF49004FEA2C1C02F5FA020CFB0EF3D7
:106E00004FEACE1E4FEA112C4FEAC1210EEB635E12
:106E100042EB22420EFB0CFC4FEA1C5300FB031119
:106E20004FEA112C4FEA01310EFB0CFC4FEADC4C0F
:106E300000FB0C11C14228BF09184CEB03335DF86D
:106E400004EB10EB410143EBC250B2F57C0F38BFAD
:106E5000704729D512F0F00F1CBF00F1C04000F0C0
:106E600000407047008182838485868788898B8C67
:106E70008D8E8F919293959697999A9C9D9FA0A2A3
:106E8000A3A5A7A8AAACAEB0B2B3B5B7B9BCBEC0F3
:106E9000C2C5C7C9CCCED1D4D7D9DCDFE2E6E9EC94
:106EA000F0F3F7FAFE0000004FEA400C0CF1807C92
:106EB000BCF17E4F28BF7047B0F1C04000F0ABB9C5
:106EC00090EA010F0CEAD11348BF42F48072624588
:106ED00038BF634507D213F47F0F16D080EA010054
:106EE00000F00040704710B500F04FF9097EFC3EFD
:106EF00000F005B880EA010000F00040704780EA29
:106F0000010000F0004000F086B912F47F0F04BFCA
:106F10000248704780EA010000F07DB90000C07FA0
:106F200050EA010C00F113801CF5000F58BFBCF5AE
:106F3000000F01D48842704707D710F5000F58BFE3
:106F400011F5000F15D488427047894270471CF52F
:106F5000000F04D5BCF5000FF7D5814270474FF004
:106F6000807C1CEB400F38BF1CEB410F01D28142EB
:106F7000704710B500F009F9922449004FF0005015
:106F80004FF08051FFF7FEBEC10DD1F19E0206DB2E
:106F90004FEA002343F0004323FA02F07047004217
:106FA00007D54FEA4001B1F1FE4F02D24FF0000089
:106FB000704710B500F0E9F849922480002070472E
:106FC0006FEA20007047000010F0004148BF4042C7
:106FD000B0FA80F310FA03F2C3F19D030BD051EA2B
:106FE000C35101EB1220530638BF704700F1010076
:106FF00008BF20F001007047B0FA80F310FA03F2E6
:10700000C3F19D030AD0D90501EB1220530638BF06
:10701000704700F1010008BF20F001007047000038
:1070200050EA010C00F113801CF5000F58BFBCF5AD
:10703000000F01D48842704707D710F5000F58BFE2
:1070400011F5000F15D488427047894270471CF52E
:10705000000F04D5BCF5000FF7D5814270474FF003
:10706000807C1CEB400F38BF1CEB410F01D28142EA
:10707000704710B500F089F8922449004FF0005095
:107080004FF08051FFF77EBE4FF47F0C1CEAD01208
:107090001EBF1CEAD11392EA0C0F93EA0C0F00F00A
:1070A000478090EA010F48BF42F480724FF0004CD5
:1070B0004CEA00204CEA012102EB0302A0FB011381
:1070C000A2F50002002918BF43F001035B0028BFAE
:1070D0004FEA330342EB22425FEA132C4CEBC250DF
:1070E0002EBFBCEB436FB2F57C0F70474FEA036CC9
:1070F000BCF1004F08BF20F00100B2F57C0F38BF93
:1071000070470BD582F0FF0212F5803FC8BF704771
:1071100000F1C040D8BF00F00040704700F5000CFF
:107120005FEA4C0C48BF7047B0F1C04000F073B844
:1071300090EA010F0CEAD11348BF42F48072624515
:1071400038BF634504D280EA010000F00040704778
:1071500010B500F01AF800BF8900013E00F007B832
:1071600000F009B85FEA410C5FEA1C6C08D080EAC5
:10717000010000F050B85FEA400C5FEA1C6CF6D1E9
:107180004FF00040A0F5800070470EF1020E2EF087
:10719000030E5EF8044B244204D44FEA4102B2F1DC
:1071A0007F4F11D84FEA4003B3F17F4F0CD80ED177
:1071B0004FEAD07CB2F17F4F0CEB4C0C0CF1020C7F
:1071C00008BF4CEBD17C04E04FF0080C01E04FEA23
:1071D000D17C0CEB4C0324FA03F404F00704B4F163
:1071E000040C06D20EEB840CBDE810404CF0010CF0
:1071F0006047DFE80CF0070802024FF00040A0F5FE
:10720000800010BD0846420018BFD2F1807288BFCE
:1072100000F0004010BDFF2141EAD050C00570478A
:1072200051EA000C00F113801CF5000F58BFBCF5AB
:10723000000F01D48142704707D711F5000F58BFE6
:1072400010F5000F15D481427047894270471CF534
:10725000000F04D5BCF5000FF7D5884270474FF0FA
:10726000807C1CEB410F38BF1CEB400F01D28842E1
:10727000704780EA010081EA000180EA0100FFF71F
:10728000F8BE000090EA010F48BF81F000413FF5D1
:1072900018AD421A04D882F00042A0EB020011445B
:1072A0004FEAD0524FF07F4C1CEA410FA2EBD15372
:1072B00018BF9CEA026F4AD04FF0004C4CEA002005
:1072C0004CEA012121FA03FCB0EB0C0C0FD412F0B4
:1072D000FE0F36D05FEA4C001DD5001240EBC250C5
:1072E00038BF70471CF03F0F18BF70470BE0A2F18A
:1072F00001025FEA1C2040EBC25038BF70471CF00F
:107300007F0F18BF7047C3F12003994014BF401E80
:1073100020F00100704780084FEA122308BF704731
:10732000B0FA80FCA2EB0C02CCF1280C60FA0CF055
:1073300093EA122F04BF00EBC25070474FEAC370AC
:107340007047130A5FEADC1008BF7047F6E79CEA53
:10735000026F04D010EA5C0F08BF0020704710B520
:10736000FFF713FF40DFF63E81F000407047F9F76A
:10737000A0B90CF00F03092B08BF082000F05180C2
:107380000A2B0BD0082B18BF704708BF1CF0400F0A
:107390000AD04FF000004FF0000170471CF0400F82
:1073A00018BF4FF0004070471CF0100F08D020F0BD
:1073B000704300F07F4242EAD3014FEA43707047C6
:1073C00000F0604021F07F4242EA000201F07F407D
:1073D00040EA727070474FF0FF0212EAD0521CBFB1
:1073E00092F0FF038B42C2BFD14200EBC150704705
:1073F000002A0AD0002B0BD0002900F00040A4BFC7
:1074000040F0FE4040F40000704700F0004070473C
:1074100043024FF00B0C18BF4CF0806C7FF4ACAC07
:1074200070471CF4801F11D01CF4E02F03D06FEACA
:10743000CC31490070474FF04050EFF3008222F00A
:10744000704242EA000282F3008870474FF0000069
:107450007047010202030405060708090A0B0C0D18
:107460000E0F1010000000000000000001020304D5
:1074700006070809000000000102030400000000E4
:1074800000000000002F00000000070007000014AB
:107490007F147F1400242A7F2A12006264081323B9
:1074A00000364955225000000503000000001C2250
:1074B0004100000041221C000014083E081400088E
:1074C000083E0808000000A060000008080808083E
:1074D000000060600000002010080402003E5149D6
:1074E000453E0000427F4000004261514946002174
:1074F00041454B31001814127F100027454545398E
:10750000003C4A49493000017109050300364949E8
:10751000493600064949291E0000363600000000A1
:1075200056360000000814224100001414141414EC
:107530000000412214080002015109060032495995
:10754000513E007C1211127C007F49494936003EB1
:1075500041414122007F4141221C007F494949416C
:10756000007F09090901003E4149497A007F080866
:10757000087F0000417F4100002040413F01007F23
:1075800008142241007F40404040007F020C027FEF
:10759000007F0408107F003E4141413E007F090901
:1075A0000906003E4151215E007F09192946004627
:1075B000494949310001017F0101003F4040403FFE
:1075C000001F2040201F003F4038403F0063140848
:1075D0001463000708700807006151494543000023
:1075E0007F41410000552A552A55000041417F0046
:1075F000000402010204004040404040000001023B
:107600000400002054545478007F48444438003823
:107610004444442000384444487F003854545418AB
:1076200000087E0901020018A4A4A47C007F0804BD
:1076300004780000447D4000004080847D00007F8D
:10764000102844000000417F4000007C04180478AA
:10765000007C0804047800384444443800FC2424A6
:1076600024180018242418FC007C0804040800488E
:107670005454542000043F444020003C4040207CAF
:10768000001C2040201C003C4030403C004428109E
:107690002844001CA0A0A07C004464544C44141452
:1076A000141414140000000000000000000000008A
:1076B00000000000000000F800000000000000339F
:1076C0003000000000100C06100C06000000000046
:1076D0000000000040C07840C0784000043F04042F
:1076E0003F040400007088FC08300000001820FFF0
:1076F000211E0000F008F000E018000000211C032B
:107700001E211E0000F00888700000001E212324A6
:107710001927211010160E000000000000000000C4
:1077200000000000000000E0180402000000000754
:107730001820400000020418E0000000004020185B
:1077400007000000404080F0804040000202010F2E
:1077500001020200000000F0000000000101011F12
:1077600001010100000000000000000080B0700076
:107770000000000000000000000000000001010106
:107780000101010100000000000000000030300095
:10779000000000000000000080601804006018066F
:1077A0000100000000E010080810E000000F1020A9
:1077B00020100F00001010F8000000000020203FF3
:1077C000202000000070080808887000003028247D
:1077D000222130000030088888483000001820201E
:1077E00020110E000000C02010F800000007042443
:1077F000243F240000F80888880808000019212088
:1078000020110E0000E0108888180000000F1120E1
:1078100020110E0000380808C83808000000003F9A
:10782000000000000070880808887000001C2221F9
:1078300021221C0000E010080810E00000003122A6
:1078400022110F00000000C0C00000000000003046
:107850003000000000000080000000000000806098
:107860000000000000008040201008000001020419
:107870000810200040404040404040000404040400
:1078800004040400000810204080000000201008BC
:1078900004020100007048080808F00000000030F1
:1078A00036010000C030C828E810E000071827247F
:1078B00023140B000000C038E0000000203C23022D
:1078C0000227382008F8888888700000203F202090
:1078D00020110E00C03008080808380007182020C2
:1078E0002010080008F808080810E000203F2020B9
:1078F00020100F0008F88888E8081000203F20209A
:107900002320180008F88888E8081000203F20008D
:1079100003000000C03008080838000007182020C5
:10792000221E020008F808000008F808203F210184
:1079300001213F20000808F8080800000020203F2F
:107940002020000000000808F8080800C08080809F
:107950007F00000008F888C028180800203F200198
:107960002638200008F8080000000000203F2020F2
:107970002020300008F8F800F8F80800203F003F09
:10798000003F200008F830C00008F808203F200021
:1079900007183F00E01008080810E0000F10202032
:1079A00020100F0008F808080808F000203F210107
:1079B00001010000E01008080810E0000F1824245E
:1079C00038504F0008F8888888887000203F2000D1
:1079D000030C302000708808080838000038202187
:1079E00021221C00180808F8080818000000203F91
:1079F0002000000008F808000008F808001F2020F8
:107A000020201F000878880000C8380800000738C8
:107A10000E010000F80800F80008F800033C070019
:107A2000073C0300081868808068180820302C0381
:107A3000032C30200838C800C83808000000203F58
:107A40002000000010080808C83808002038262147
:107A500020201800000000FE020202000000007F4B
:107A600040404000000C30C0000000000000000159
:107A70000638C00000020202FE0000000040404044
:107A80007F00000000000402020204000000000069
:107A900000000000000000000000000080808080E6
:107AA00080808080000202040000000000000000CE
:107AB0000000000000008080808000000019242267
:107AC00022223F2008F8008080000000003F1120A3
:107AD00020110E000000008080800000000E1120A8
:107AE00020201100000000808088F800000E112086
:107AF00020103F200000808080800000001F222294
:107B000022221300008080F0888888180020203FFF
:107B1000202000000000808080808000006B949412
:107B20009493600008F8008080800000203F2100CE
:107B300000203F2000809898000000000020203F97
:107B400020200000000000809898000000C0808085
:107B5000807F000008F8000080808000203F240221
:107B60002D302000000808F8000000000020203F11
:107B7000202000008080808080808000203F2000C6
:107B80003F20003F8080008080800000203F210057
:107B900000203F200000808080800000001F202007
:107BA00020201F00808000808000000080FFA12036
:107BB00020110E000000008080808000000E112047
:107BC00020A0FF80808080008080800020203F21D6
:107BD0002000010000008080808080000033242489
:107BE00024241900008080E0808000000000001F35
:107BF000202000008080000000808000001F2020E6
:107C000020103F20808080000080808000010E30A6
:107C10000806010080800080008080800F300C0307
:107C20000C300F0000808000808080000020312E0A
:107C30000E312000808080000080808080818E70E6
:107C40001806010000808080808080000021302C98
:107C50002221300000000000807C020200000000B1
:107C6000003F404000000000FF0000000000000056
:107C7000FF0000000002027C800000000040403F46
:107C800000000000000601010202040400000000E0
:107C90000000000002400000000000A00000000002
:107CA00005400000000000C8000000000C4000007B
:107CB0000000409C00000000194000000020BCBEF5
:107CC0000000000034400000BFC91B8E000000040B
:107CD000B5400000504BCFD06607E2CF0100000056
:107CE0006C4100003E8251AADFEEA7340100000083
:107CF000D9420000DCB5A0E23A301F97FFFFFFFF3A
:107D0000B4450000FD25A0C8E9A3C14FFFFFFFFF58
:107D1000FF3F00000000008000000000FF3F000067
:107D20000000008000000000647D000800000020CA
:107D3000640100006C010008A47D000864010020BB
:107D400034090000A80100081C00000043000000E6
:107D5000F8FFFFFF0C0000000E0000000F00000005
:107D60002E000000014542019210C324F4337041FB
:107D700093A54408160501000A000AFF021001330A
:107D8000204E33409C33DC0533E80333B80B034704
:107D9000D00742010228010214018201E201041805
:047DA000A100B1008D
:0400000508000131BD
:00000001FF
